:1062FB00E5467006127B658F4622E546B40506120D
:10630B003B738F4622E546B40B061271718F462202
:10631B00E546B40A061268568F4622E546B40F06C8
:10632B00126C618F4622E546B414061265078F4640
:10633B0022E546B41906127AA88F4622E546B41E0A
:10634B0006127B798F4622E546B42306126CB78F73
:10635B004622E546B42806127C2E8F4622E546B42B
:10636B002D06127B8D8F4622E546B4320512741230
:03637B008F462228
:107B6500C20890061EE0FFA3E0901CECCFF0A3EF47
:047B7500F07F052276
:103B7300127C2A50477D047F011262735008E53E90
:103B8300B401037F0B227D047F021262735008E5A8
:103B93003EB402037F0B227D047F0312627350083D
:103BA300E53EB403037F0B227D047F04126273504E
:103BB30008E53EB404037F0B227F0A227F081275B7
:103BC300F650061253747F00227D057F051262733F
:103BD3005032901CEEE07002A3E070282046257D51
:103BE300017F011262734003023CE990066CE0FF1F
:103BF3007C0A7D70127357900610E0FFA3E0901CBF
:103C0300EE023CB07D067F051262735031901CF0CA
:103C1300E07002A3E070272048247D017F02126236
:103C2300734003023CE990066DE0FF7C0A7D90122D
:103C33007357900612E0FFA3E0901CF0806F7D079E
:103C43007F051262735031901CF2E07002A3E070A2
:103C530027204C247D017F031262734003023CE959
:103C630090066EE0FF7C0A7DB0127357900614E055
:103C7300FFA3E0901CF280357D087F05126273502C
:103C830033901CF4E07002A3E07029204F267D01DD
:103C93007F04126273504F90066FE0FF7C0A7DD061
:103CA300127357900616E0FFA3E0901CF4CFF0A325
:103CB300EFF080327D077F06126273500F30290CBC
:103CC300901CECE07002A3E07002C22930380C9023
:103CD3001CECE07002A3E07002C238786CE6B40515
:093CE300057F04125DBF7F05227C
:10717100203842900633E0901D10F0123346E53E70
:10718100B401062049247F0522E53EB40206204DC4
:10719100197F0522E53EB4030620510E7F0522E545
:1071A1003EB404062054037F0522901D10E0D394C1
:0871B1000050C8D2387F0A2209
:10685600E53B700AE53EB40105753B018028E53B42
:10686600700AE53EB40205753B02801AE53B700AE4
:10687600E53EB40305753B03800CE53B7008E53E39
:10688600B40403753B047D077F06126273500C7DCA
:10689600077F06126273501E30291B900650E0FFD8
:1068A6007C067DF01273577D017F011262735006DC
:0968B600120FB3122B647F0F22B4
:106C6100127C2A503F120FB3202F09203006203109
:106C710003303209E53270051277BA800B786CE681
:106C8100B4050B7F03125DBF122B64120FB3202FCB
:106C91001020300D20310A203207E5327003122B0B
:106CA100647F0F221277BA7D057F0712627350034A
:066CB1007F14227F002287
:10650700E4F53B7D077F06126273500C7D077F061B
:10651700126273505E30295B786CE670047F0180ED
:1065270008786CE6B404077F02125DBF8038786C88
:10653700E6B407047601802E7D037F05126273504F
:1065470025901CF6E07002A3E0701B900662E0FF46
:106557007C097D30127357900620E0FFA3E0901C62
:10656700F6CFF0A3EFF07F061275F650037F0022F7
:106577007F19227D077F0612627350052029027F4B
:026587000522EB
:107AA8007D077F0612627350062029037F05229006
:0A7AB8000630E0901D10F07F1E2242
:107B7900901D10E070037F2322127C2A50037F0A94
:047B8900227F1E2217
:106CB7007D047F071262735041E53EB4010B9006D5
:106CC7005EE0FF7C087DB0802EE53EB4020B9006A7
:106CD7005FE0FF7C087DD0801EE53EB4030B900685
:106CE70060E0FF7C087DF0800EE53EB4040C900662
:106CF70061E0FF7C097D10127357900631E0901D0B
:056D070010F07F2822BE
:037C2E007F2D2285
:107B8D00901D10E070037F3222127C2A50037F0A71
:047B9D00227F2D22F4
:107412003058037F32227D047F0512627350289018
:107422001CF8E07002A3E0701E900663E0FF7C0986
:107432007D50127357900622E0FFA3E0901CF8CF14
:0C744200F0A3EFF07F3222C2087F00228E
:1072D400900640E06035D259D224753D03123346FE
:1072E400122B64120FB3127C2A5009E53D6005127B
:1072F400334680F2E4F522F523127C2A4009E53D69
:10730400600512334680F2E53D70D2C259C224C2F0
:027314005822FD
:04000E0001000530B8
:0300030002698708
:0B698700C0E0C083C082C0D075D00803
:10699200853082852F83E493FF204404C4540FFF83
:1069A200430FF08F80C284D28500C2870000D28755
:1069B200007580FF7580FEC284C28500C287000018
:1069C2000000D287007580FF30440CC2440530E5D8
:0B69D200307006052F8002D244D2A8CE
:0969DD00D0D0D082D083D0E0328A
:03000B00021BB61F
:101BB600C0E0C0F0C083C082C0D075D008758CD894
:101BC600758A92D28C12433B12755BE531D3940031
:101BD60040051531021F40753111901D10E0D39458
:101BE600004003E014F0901D11E0D394004003E0A0
:101BF60014F0901D12E0D394004003E014F0901D01
:101C060013E0D394004003E014F0E532D39400408F
:101C16000215321541E541B40A004003021F3D900A
:101C26001C2CF8282873021F40021E91021E59021E
:101C36001E2C021DC2021D58021CEE021C84021C30
:101C460067021C4AD3901CEDE09400901CECE094D3
:101C5600005003021F40A3E024FFF0901CEC021F7B
:101C660031D3901CE9E09400901CE8E09400500306
:101C7600021F40A3E024FFF0901CE8021F317F0101
:101C86001278824003021F40901CE1E09400901CF1
:101C9600E0E09400400CA3E024FFF0901CE0E03468
:101CA600FFF0D3901CEFE09400901CEEE09400400F
:101CB6000CA3E024FFF0901CEEE034FFF0D3901C60
:101CC600FBE09400901CFAE094005003021F407D54
:101CD600067F011262734003021F40901CFBE02442
:101CE600FFF0901CFA021F317F0212788240030235
:101CF6001F40901CE3E09400901CE2E09400400C2E
:101D0600A3E024FFF0901CE2E034FFF0D3901CF136
:101D1600E09400901CF0E09400400CA3E024FFF057
:101D2600901CF0E034FFF0D3901CFDE09400901C72
:101D3600FCE094005003021F407D067F021262738E
:101D46004003021F40901CFDE024FFF0901CFC02A3
:101D56001F317F031278824003021F40901CE5E08A
:101D66009400901CE4E09400400CA3E024FFF09063
:101D76001CE4E034FFF0D3901CF3E09400901CF2D6
:101D8600E09400400CA3E024FFF0901CF2E034FF46
:101D9600F0D3901CFFE09400901CFEE094005003EA
:101DA600021F407D067F031262734003021F4090AC
:101DB6001CFFE024FFF0901CFE021F317F04127806
:101DC600824003021F40901CE7E09400901CE6E06E
:101DD6009400400CA3E024FFF0901CE6E034FFF0F2
:101DE600D3901CF5E09400901CF4E09400400CA302
:101DF600E024FFF0901CF4E034FFF0D3901D01E0E6
:101E06009400901D00E094005003021F407D067F61
:101E1600041262734003021F40901D01E024FFF08C
:101E2600901D00021F31D3901CEBE09400901CEA39
:101E3600E09400400CA3E024FFF0901CEAE034FF9D
:101E4600F0901D14E0D394005003021F40E014F0FC
:101E5600021F40D3901CF9E09400901CF8E0940017
:101E6600400CA3E024FFF0901CF8E034FFF0D39080
:101E76001CF7E09400901CF6E094005003021F400B
:101E8600A3E024FFF0901CF6021F31786CE6FF7089
:101E960003021F40EFB401059006188027786CE610
:101EA600FFB40219D3901CEBE09400901CEAE09476
:101EB60000403FA3E024FFF0901CEA806EEFB403DD
:101EC6001190061AE0FFA3E0901CEACFF0A3EFF012
:101ED6008020786CE6FFB4041ED3901CEBE09400DF
:101EE600901CEAE09400400AA3E024FFF0901CEA6C
:101EF6008039786C068043EF6405603E786CE6FFB7
:101F0600B4060D901CEA7402F0A37458F006802AF9
:101F1600EFB40726D3901CEBE09400901CEAE09403
:101F260000400EA3E024FFF0901CEAE034FFF080AE
:101F360009786C7600800375410A127A55400812BA
:101F460076884003127A71D0D0D082D083D0F0D078
:021F5600E03277
:0300130002615B2C
:0D615B00C0E0C0F0C083C082C0D075D0107D
:1061680075A0FFC284C285D287C286308018C2A4B7
:10617800C2A5D2A6C2A7E5A0540FF54AD2A7FF121E
:106188006609D286804F308118D2A4C2A5D2A6C291
:10619800A7E5A0540FF54AD2A7FF12637ED28680E6
:1061A80034308218C2A4D2A5D2A6C2A7E5A0540F43
:1061B800F54AD2A7FF126401D2868019308316D21D
:1061C800A4D2A5D2A6C2A7E5A0540FF54AD2A7FF2C
:0561D800126484D28670
:0B61DD00D0D0D082D083D0F0D0E032D0
:106C0A00BF0113900632E0901D10F0901D10E0D3E2
:106C1A009400404280F5BF0213900632E0901D11A5
:106C2A00F0901D11E0D39400402C80F5BF0313901F
:106C3A000632E0901D12F0901D12E0D39400401627
:106C4A0080F5BF0411900632E0901D13F0901D13D9
:076C5A00E0D3940050F72283
:106D0C00304712205F0F900672E0FF7C0B7D301233
:106D1C007357D25F22304B1220610F900673E0FF45
:106D2C007C0B7D50127357D26122304E1220620FB1
:106D3C00900674E0FF7C0B7D70127357D262223088
:106D4C00521120630E900675E0FF7C0B7D90127340
:046D5C0057D2632285
:10551F00303D1A204617900664E0FF7C097D70121B
:10552F007357D246C214C210C21CC218223046147E
:10553F00203911900665E0FF7C097D90127357C2E8
:10554F0046C23D22303E1A204817900666E0FF7C87
:10555F00097DB0127357D248C215C211C21DC219AC
:10556F0022304814203A11900667E0FF7C097DD065
:10557F00127357C248C23E2230401A204C17900671
:10558F0068E0FF7C097DF0127357D24CC216C2122D
:10559F00C21EC21A22304C14203B11900669E0FF44
:1055AF007C0A7D10127357C24CC2402230421A201F
:1055BF004F1790066AE0FF7C0A7D30127357D24F67
:1055CF00C217C213C21FC21B22304F13203C1090B0
:1055DF00066BE0FF7C0A7D50127357C24FC2422206
:1055EF00124221D28C7F071275F6500512001680D9
:1055FF00121272017F1F7E001278A990001FEFF028
:10560F001276E27F081275F650051259B480FE909B
:10561F0006087402F0A37458F090060A7402F0A3FF
:10562F007458F090060C7402F0A37458F090060EA4
:10563F007402F0A37458F0900681E0FF7C0D7D108A
:10564F00127357D208127A717545017F01125DBF2F
:10565F00900618E0FFA3E0901CEACFF0A3EFF0C292
:10566F0008127A71123346305A11E53EB4010C908C
:10567F000651E0FF7C077D101273571262FB305BFF
:10568F0003124566305C03124453305D031249A97F
:10569F00306003124AB3124EC27D077F0612627347
:0C56AF004002C22912551F126D0C80B879
:104566007C007D80C2677F011236B950117F06122A
:1045760075F65002D2087F01121F580246067C00CB
:104586007D70D2677F011236B95002800D7C007DA6
:1045960078D2677F011236B950077F011209418030
:1045A6005F7C007DA0D2677F011236B950117D076E
:1045B6007F0612627350087545011277E380417CCD
:1045C600007DA8C2677F011236B950197D057F01AB
:1045D60012627350107F061275F65002D2087F01E0
:1045E600124678801B7C007DB0C2677F011236B907
:1045F600500E7F061275F65002D2087F011250B295
:10460600E4F54CAF4CEF3395E0FEEF7803C333CEC1
:1046160033CED8F92400F58274013EAD82FCD26710
:104626007F011236B95038754501AF4CEF3395E02E
:10463600FE74A02FF58274063EF583E0FFC007AF37
:104646004CEF3395E0FEEF7805C333CE33CED8F981
:1046560024F0F58274103EAD82FCD007126F55052A
:104666004CC3E54C648094A84099C25BC265126D48
:0146760060E3
:014677002220
:104453007F061275F65002C2087D017F0612627351
:10446300503D7C007D88C2677F021236B9500BD263
:10447300097F02121F58C20980257C007D70D26714
:104483007F021236B95002800D7C007D78D2677F9F
:10449300021236B95009D2097F02120941C20990AA
:1044A300001FE030E1427C007DA0D2677F0212361C
:1044B300B950147D077F06126273500B1278CF75C3
:1044C30045021277E3801E7C007DA8C2677F02123B
:1044D30036B950147D057F02126273500B1278CFE8
:1044E3007F021246781279C07D027F0612627350F2
:1044F3006AE4F54CAF4CEF3395E0FEEF7803C3333A
:10450300CE33CED8F92400F58274013EAD82FCD2BD
:10451300677F021236B95038754502AF4CEF3395B9
:10452300E0FE74A02FF58274063EF583E0FFC0071A
:10453300AF4CEF3395E0FEEF7805C333CE33CED8DF
:10454300F924F0F58274103EAD82FCD007126F554A
:10455300054CC3E54C648094A84099C25CC26612C2
:024563006DB435
:014565002233
:1049A9007D037F06126273503D7C007D90C2677F54
:1049B900031236B9500BD20E7F03121F58C20E8054
:1049C900257C007D70D2677F031236B95002800DB5
:1049D9007C007D78D2677F031236B95009D20E7FE9
:1049E90003120941C20E90001FE030E2427C007DB3
:1049F900A0D2677F031236B950147D077F06126271
:104A090073500B1278CF7545031277E3801E7C0033
:104A19007DA8C2677F031236B950147D057F031242
:104A29006273500B1278CF7F031246781279C07DDA
:104A3900047F06126273506AE4F54CAF4CEF33956C
:104A4900E0FEEF7803C333CE33CED8F92400F582E4
:104A590074013EAD82FCD2677F031236B9503875B6
:104A69004503AF4CEF3395E0FE74A02FF582740631
:104A79003EF583E0FFC007AF4CEF3395E0FEEF78DA
:104A890005C333CE33CED8F924F0F58274103EAD88
:104A990082FCD007126F55054CC3E54C648094A87D
:094AA9004099C25DC228126E089A
:014AB20022E1
:104AB3007D057F06126273503D7C007D98C2677F3F
:104AC300041236B9500BD20C7F04121F58C20C804B
:104AD300257C007D70D2677F041236B95002800DA9
:104AE3007C007D78D2677F041236B95009D20C7FDF
:104AF30004120941C20C90001FE030E3427C007DA8
:104B0300A0D2677F041236B950147D077F06126264
:104B130073500B1278CF7545041277E3801E7C0027
:104B23007DA8C2677F041236B950147D057F041235
:104B33006273500B1278CF7F041246781279C07DCE
:104B4300067F06126273506AE4F54CAF4CEF33955F
:104B5300E0FEEF7803C333CE33CED8F92400F582D9
:104B630074013EAD82FCD2677F041236B9503875AA
:104B73004504AF4CEF3395E0FE74A02FF582740625
:104B83003EF583E0FFC007AF4CEF3395E0FEEF78CF
:104B930005C333CE33CED8F924F0F58274103EAD7D
:104BA30082FCD007126F55054CC3E54C648094A872
:094BB3004099C260C22A126E5C36
:014BBC0022D6
:106FF500BF010AC214C210C21CC2188025BF020AF2
:10700500C215C211C21DC2198018BF030AC216C219
:1070150012C21EC21A800BBF0408C217C213C21FB8
:10702500C21B90001FE0FF30E002D224EF30E102E6
:0E703500D225EF30E202D226EF30E302D2275E
:01704300222A
:106609008F4B7868E6C39450507130496E20596BAE
:106619007D077F01126273502B205E287868E6702F
:106629000D90063BE0B54B06203F03D23F22202FB9
:106639000D203F0A7F01126FF5753D02D22F90069A
:1066490034E0F5327D087F06126273501990063FD7
:10665900E0B54B06205E03D265220534E534AE333E
:10666900700E0533800A0534E534AE337002053304
:0C66790014F5828E83E54BF07868062251
:10637E008F4B7869E6C394505078304D7520597222
:10638E007D077F0212627350327F02127882502B89
:10639E00205E287869E6700D90063BE0B54B06202E
:1063AE004103D2412220300D20410A7F02126FF5A7
:1063BE00753D02D230900634E0F5327D087F06122C
:1063CE006273501990063FE0B54B06205E03D2660D
:1063DE00220536E536AE35700E0535800A0536E5F2
:1063EE0036AE357002053514F5828E83E54BF078A6
:0363FE006906220B
:106401008F4B786AE6C39450507830517520597299
:106411007D077F0312627350327F03127882502B03
:10642100205E28786AE6700D90063BE0B54B0620A9
:106431004303D2432220310D20430A7F03126FF51B
:10644100753D02D231900634E0F5327D087F0612A7
:106451006273501990063FE0B54B06205E03D228C7
:10646100220538E538AE37700E0537800A0538E564
:1064710038AE377002053714F5828E83E54BF0781C
:036481006A062286
:106484008F4B786BE6C39450507830547520597212
:106494007D077F0412627350327F04127882502B7E
:1064A400205E28786BE6700D90063BE0B54B062025
:1064B4004503D2452220320D20450A7F04126FF590
:1064C400753D02D232900634E0F5327D087F061223
:1064D4006273501990063FE0B54B06205E03D22A42
:1064E40022053AE53AAE39700E0539800A053AE5D7
:1064F4003AAE397002053914F5828E83E54BF07893
:036504006B062201
:1078CF0090001FE0FF30E004D208D220EF30E10437
:1078DF00D209D221EF30E204D20ED222EF30E304EC
:0578EF00D20CD223229F
:1079C000C220C221C222C22390001FE0FF30E10288
:0F79D000C209EF30E202C20EEF30E302C20C2216
:105DBF008F4C304603025E5B304803025E5B304C13
:105DCF0003025E5B304F03025E5B7D017F01126257
:105DDF00735079E54CB401197D017F051262735040
:105DEF000C90065AE0FF7C087D30127357786C06D2
:105DFF0022E54CB402177D027F0512627350489062
:105E0F00065BE0FF7C087D50127357803AE54CB477
:105E1F00041A7D027F05126273500C90065DE0FF3D
:105E2F007C087D90127357786C760622E54C6403DC
:105E3F00701E7D027F05126273500C90065CE0FFAE
:105E4F007C087D70127357786C760122E4786CF6BB
:015E5F002220
:107A8D00EF1FAA0670011ED39400EA9400400BE488
:0A7A9D00FDEDC394C850E90D80F719
:017AA70022BC
:105A69008F5D306B5BE55DB40111D22090001FE0C2
:105A7900F420E003305E44D2088040E55DB40211B1
:105A8900D22190001FE0F420E103305E2ED209807C
:105A99002AE55DB40311D22290001FE0F420E2034D
:105AA900305E18D20E8014E55DB4040FD223900045
:105AB9001FE0F420E303305E02D20CAF5D026C0AF2
:105AC900E55DB40110C22090001FE0F420E003302E
:105AD9005E41C20822E55DB40210C22190001FE0B8
:105AE900F420E103305E2CC20922E55DB40310C243
:105AF9002290001FE0F420E203305E17C20E22E577
:105B09005DB4040FC22390001FE0F420E303305E6C
:045B190002C20C2296
:105B1D008F5330695BE553B40111D22490001FE01F
:105B2D00F420E003305E44D2088040E553B4021106
:105B3D00D22590001FE0F420E103305E2ED20980C3
:105B4D002AE553B40311D22690001FE0F420E2039E
:105B5D00305E18D20E8014E553B4040FD227900096
:105B6D001FE0F420E303305E02D20CAF53026C0A47
:105B7D00E553B40110C22490001FE0F420E003307F
:105B8D005E41C20822E553B40210C22590001FE009
:105B9D00F420E103305E2CC20922E553B40310C298
:105BAD002690001FE0F420E203305E17C20E22E5BE
:105BBD0053B4040FC22790001FE0F420E303305EBE
:045BCD0002C20C22E2
:08290E008F538C548D558B563C
:10291600C267E55524FFF582E55434FFF583E0F5FB
:1029260058855582855483E0FFF559A3E0FEF55A94
:10293600EF14B40800505C90294B75F003A4C583CE
:1029460025F0C5837302296302296A0229710229C7
:102956007802297F02298602298D0229947557015A
:10296600D267802F755702D2678028755704D267C1
:102976008021755708D267801A755710D267801361
:10298600755720D267800C755740D26780057557FA
:1029960080D267EE24FE7003022A5B24F8605C2472
:1029A600096003022A6DE553B401059000208045B5
:1029B600E553B40205900021803BE553B40305902E
:1029C60000228031E553B404059000238027E553A7
:1029D600B40505900024801DE553B4060590002536
:1029E6008013E553B407059000268009E553640873
:1029F6007077900027E04557F0806EE553B40105E7
:102A06009000208045E553B40205900021803BE507
:102A160053B403059000228031E553B404059000B9
:102A2600238027E553B40505900024801DE553B4A3
:102A360006059000258013E553B40705900026800F
:102A460009E55364087022900027E0FFE557F4FE7D
:102A5600EF5EF08014E553B4080D855582855483E6
:102A6600E0FF1260C7C267C267206703022B63E5F7
:102A760053B40109900020E0FD7F208060E553B447
:102A86000209900021E0FD7F218052E553B403093D
:102A9600900022E0FD7F228044E553B404099000B3
:102AA60023E0FD7F238036E553B40509900024E03A
:102AB600FD7F248028E553B40609900025E0FD7FBC
:102AC60025801AE553B40709900026E0FD7F26808D
:102AD6000CE553B4080C900027E0FD7F277E00121A
:102AE6007397D2AFD26BAF56125A69AD58E4FF1244
:102AF6007766AD59E4FF127766E55AB401047D386E
:102B06008007E55AB40A077D367F06127766E553D5
:102B1600B408031276E27D077F06126273500B201B
:102B26002908C208C209C20EC20C7D017F011262C9
:102B3600734002C2087D017F021262734002C2091D
:102B46007D017F031262734002C20E7D017F041273
:0D2B560062734002C20CC26BAF56125A6986
:012B6300224F
:045E60008F538D547B
:105E6400D26BAF54125A69AF54126C0AE553B401A1
:105E7400059000208044E553B40205900021803A47
:105E8400E553B403059000228030E553B404059033
:105E940000238026E553B40505900024801CE553B7
:105EA400B406059000258012E553B407059000263A
:105EB4008008E553B40806900027E0F555E55560E1
:105EC40025755701E4F556E55530E007AD57E4FF75
:105ED400127766E555C313F55505570556E556C3C0
:105EE400940840E3800E7D187F021277667D537F0D
:0B5EF40002127766C26BAF54125A69AD
:015EFF002280
:021F58008F4DAB
:101F5A00E54D6401701E754E1B754F10900080E0B0
:101F6A00F550E54F2550F582E4354EF583E0F552FC
:101F7A0078688069E54D6402701E754E1B754F6066
:101F8A00900088E0F550E54F2550F582E4354EF58E
:101F9A0083E0F55278698045E54D6403701E754EFD
:101FAA001B754FB0900090E0F550E54F2550F58233
:101FBA00E4354EF583E0F552786A8021E54DB404A4
:101FCA001F754E1C754F00900098E0F550E54F259F
:101FDA0050F582E4354EF583E0F552786BE6F5511B
:101FEA00E55214B4090040030222F790200375F069
:101FFA0003A4C58325F0C5837302201E0220710243
:10200A0020C402211702216A0221BD0222100222E3
:10201A00610222B1E54F2550F582E4354EF583A3DE
:10202A00E0B40A18E5502402FFE433FEE551B5078F
:10203A000BE4B50607AD4D7F01022286AF507E0044
:10204A00EF2403FDEE33FCE5516D7001EC600302F1
:10205A0022F7EF254FFFEE354ECF2401FDE43FFC7A
:10206A00AB4D7F010222AEE54F2550F582E4354E95
:10207A00F583A3E0B40A18E5502402FFE433FEE531
:10208A0051B5070BE4B50607AD4D7F02022286AFB4
:10209A00507E00EF2403FDEE33FCE5516D7001EC38
:1020AA0060030222F7EF254FFFEE354ECF2401FDE4
:1020BA00E43FFCAB4D7F020222AEE54F2550F5828C
:1020CA00E4354EF583A3E0B40A18E5502402FFE490
:1020DA0033FEE551B5070BE4B50607AD4D7F0302A4
:1020EA002286AF507E00EF2403FDEE33FCE5516DEE
:1020FA007001EC60030222F7EF254FFFEE354ECF59
:10210A002401FDE43FFCAB4D7F030222AEE54F25DF
:10211A0050F582E4354EF583A3E0B40A18E550245D
:10212A0002FFE433FEE551B5070BE4B50607AD4DF2
:10213A007F04022286AF507E00EF2403FDEE33FCBB
:10214A00E5516D7001EC60030222F7EF254FFFEEB7
:10215A00354ECF2401FDE43FFCAB4D7F040222AE95
:10216A00E54F2550F582E4354EF583A3E0B40A180D
:10217A00E5502402FFE433FEE551B5070BE4B5064A
:10218A0007AD4D7F05022286AF507E00EF2403FD86
:10219A00EE33FCE5516D7001EC60030222F7EF2586
:1021AA004FFFEE354ECF2401FDE43FFCAB4D7F05DA
:1021BA000222AEE54F2550F582E4354EF583A3E0C1
:1021CA00B40A18E5502402FFE433FEE551B5070BC3
:1021DA00E4B50607AD4D7F06022286AF507E00EFBA
:1021EA002403FDEE33FCE5516D7001EC600302221D
:1021FA00F7EF254FFFEE354ECF2401FDE43FFCAB50
:10220A004D7F060222AEE54F2550F582E4354EF5A4
:10221A0083A3E0B40A17E5502402FFE433FEE55134
:10222A00B5070AE4B50606AD4D7F07804FAF507E6D
:10223A0000EF2403FDEE33FCE5516D7001EC600301
:10224A000222F7EF254FFFEE354ECF2401FDE43F82
:10225A00FCAB4D7F07804DE54F2550F582E4354EA6
:10226A00F583A3E0B40A18E5502402FFE433FEE53F
:10227A0051B5070BE4B50607AD4D7F08025E60AFA6
:10228A00507E00EF2403FDEE33FCE5516D7001EC46
:10229A00705BEF254FFFEE354ECF2401FDE43FFC86
:1022AA00AB4D7F0802290EE54F2550F582E4354EE5
:1022BA00F583A3A3E07036E54F2550F582E4354E49
:1022CA00F583A3E024F96008147022AF4D02785B0D
:1022DA00D26B7F01125A69AF4D126C0A7D5E7F0282
:0D22EA00127766C26B7F01125A691259B457
:0122F70022C4
:0436B9008C4D8D4E59
:1036BD00054EE54E7002054D14F5828C83E0F970D0
:1036CD000302385BBF010875331B753410801FBFB3
:1036DD00020875351B7536608014BF030875371BDE
:1036ED007538B08009BF040675391C753A0020671E
:1036FD00030237C1BF01087868E6696002C322BFC3
:10370D0002087869E6696002C322BF0308786AE699
:10371D00696002C322BF0408786BE6696002C322A8
:10372D00E4FEEEC39940030237BFEF6401701CE560
:10373D004E2EF582E4354DF583E0FDE5342EF58210
:10374D00E43533F583E06D6002C322EF6402701C33
:10375D00E54E2EF582E4354DF583E0FDE5362EF58B
:10376D0082E43535F583E06D6002C322EF640370AA
:10377D001CE54E2EF582E4354DF583E0FDE5382E42
:10378D00F582E43537F583E06D6002C322EF640402
:10379D00701CE54E2EF582E4354DF583E0FDE53ADE
:1037AD002EF582E43539F583E06D6002C3220E02F9
:1037BD00372FD32230670302385CE4FEEEC3994005
:1037CD0003023859EF6401701CE54E2EF582E43585
:1037DD004DF583E0FDE5342EF582E43533F583E0D8
:1037ED006D6065C322EF6402701CE54E2EF582E418
:1037FD00354DF583E0FDE5362EF582E43535F5835F
:10380D00E06D6044C322EF6403701CE54E2EF5821B
:10381D00E4354DF583E0FDE5382EF582E43537F5D9
:10382D0083E06D6023C322EF6404701CE54E2EF51A
:10383D0082E4354DF583E0FDE53A2EF582E4353928
:0F384D00F583E06D6002C3220E0237C9D322C398
:01385C002249
:102B640090001FE0540FF55CB4010BE53EB4010383
:102B7400D21422C21422E55C6403702AE53EB40137
:102B840006D214D2108004C214C210E53EB402115D
:102B9400D2157D017F071262734003022D7FD2118B
:102BA40022C215C21122E55C6405702AE53EB40117
:102BB40006D214D21C8004C214C21CE53EB4031114
:102BC400D2167D027F071262734003022D7FD21E4C
:102BD40022C216C21E22E55C6409702AE53EB401D5
:102BE40006D214D2188004C214C218E53EB40411EB
:102BF400D2177D037F071262734003022D7FD21B1D
:102C040022C217C21B22E55C6407704EE53EB40184
:102C140008D214D210D21C8006C214C210C21CE501
:102C24003EB40211D2157D017F071262735002D2A5
:102C340011D21D8006C215C211C21DE53EB4031394
:102C4400D216D2127D027F071262734003022D7FD7
:102C5400D21E22C216C212C21E22E55C640B704E42
:102C6400E53EB40108D214D210D2188006C214C2B0
:102C740010C218E53EB40211D2157D017F0712621D
:102C8400735002D211D2198006C215C211C219E5BD
:102C94003EB40413D217D2137D037F07126273402C
:102CA40003022D7FD21B22C217C213C21B22E55C72
:102CB400640D704BE53EB40108D214D21CD21880C6
:102CC40006C214C21CC218E53EB40311D2167D021A
:102CD4007F071262735002D21ED21A8006C216C235
:102CE4001EC21AE53EB40413D217D21F7D037F0718
:102CF4001262734003022D7FD21B22C2178078E533
:102D04005C640F7076E53EB4010AD214D210D21C72
:102D1400D2188008C214C210C21CC218E53EB40204
:102D240013D2157D017F071262735002D211D21D96
:102D3400D2198008C215C211C21DC219E53EB403DE
:102D440013D216D2127D027F071262735002D21E72
:102D5400D21A8008C216C212C21EC21AE53EB404B8
:102D640012D217D213D21F7D037F07126273500B46
:0B2D7400D21B22C217C213C21FC21BD9
:012D7F002231
:100FB30090001FE0540FF55CB401167D017F011210
:100FC3006273500A7F061275F64003D20822C208E4
:100FD30022E55C6403705BE53E640170257D017F5F
:100FE30001126273500B7F061275F64004D208801B
:100FF30002C2087D017F021262735003D20922C22A
:101003000922E53E640260030214637D017F01123D
:1010130062735004D2088002C2087D017F0212620B
:1010230073500C7D017F071262735003D20922C2F1
:101033000922E55C6405705BE53E640170257D0172
:101043007F01126273500B7F061275F64004D208BB
:101053008002C2087D017F031262735003D20E2205
:10106300C20E22E53E640360030214637D017F0127
:101073001262735004D2088002C2087D017F0312FA
:101083006273500C7D027F071262735003D20E22EB
:10109300C20E22E55C6409705BE53E640170257D48
:1010A300017F01126273500B7F061275F64004D262
:1010B300088002C2087D017F041262735003D20CC0
:1010C30022C20C22E53E640460030214637D017FA7
:1010D300011262735004D2088002C2087D017F04AA
:1010E300126273500C7D037F071262735003D20C9C
:1010F30022C20C22E55C640760030211B5E53E647D
:101103000170347D017F01126273500B7F061275EB
:10111300F64004D2088002C2087D017F0212627386
:101123005004D2098002C2097D017F031262735009
:1011330003D20E22C20E22E53E640270367D017F89
:10114300011262735004D2088002C2087D017F023B
:10115300126273500D7D017F071262735004D2092E
:101163008002C2097D017F031262735003D20E22F3
:10117300C20E22E53E640360030214637D017F0116
:101183001262735004D2088002C2087D017F0212EA
:1011930062735004D2098002C2097D017F03126287
:1011A30073500C7D027F071262735003D20E22C26A
:1011B3000E22E55C640B6003021273E53E6401706A
:1011C300347D017F01126273500B7F061275F64066
:1011D30004D2088002C2087D017F021262735004A8
:1011E300D2098002C2097D017F041262735003D2C7
:1011F3000C22C20C22E53E640270367D017F01128F
:1012030062735004D2088002C2087D017F02126219
:1012130073500D7D017F071262735004D20980025F
:10122300C2097D017F041262735003D20C22C20CE7
:1012330022E53E640460030214637D017F011262B0
:10124300735004D2088002C2087D017F02126273C8
:101253005004D2098002C2097D017F0412627350D7
:101263000C7D037F071262735003D20C22C20C223F
:10127300E55C640D6003021331E53E640170347D67
:10128300017F01126273500B7F061275F64004D280
:10129300088002C2087D017F031262735004D20EDC
:1012A3008002C20E7D017F041262735003D20C22AE
:1012B300C20C22E53E640370367D017F0112627326
:1012C3005004D2088002C2087D017F03126273506A
:1012D3000D7D027F071262735004D20E8002C20E8C
:1012E3007D017F041262735003D20C22C20C22E5EB
:1012F3003E640460030214637D017F011262735034
:1013030004D2088002C2087D017F03126273500475
:10131300D20E8002C20E7D017F04126273500C7DD7
:10132300037F071262735003D20C22C20C22E55CC6
:10133300640F6003021463E53E640170437D017F23
:1013430001126273500B7F061275F64004D20880B7
:1013530002C2087D017F021262735004D209800227
:10136300C2097D017F031262735004D20E8002C250
:101373000E7D017F041262735003D20C22C20C2231
:10138300E53E640270457D017F011262735004D211
:10139300088002C2087D017F02126273500D7D0135
:1013A3007F071262735004D2098002C2097D017F54
:1013B300031262735004D20E8002C20E7D017F04B9
:1013C3001262735003D20C22C20C22E53E640370F6
:1013D300457D017F011262735004D2088002C20866
:1013E3007D017F021262735004D2098002C2097D1B
:1013F300017F03126273500D7D027F0712627350E7
:1014030004D20E8002C20E7D017F04126273500368
:10141300D20C22C20C22E53E640470447D017F019C
:101423001262735004D2088002C2087D017F021247
:1014330062735004D2098002C2097D017F031262E4
:10144300735004D20E8002C20E7D017F04126273B8
:10145300500C7D037F071262735003D20C22C20C1F
:011463002266
:10795F007F011278825010C209C20EC20C7F06122C
:10796F0075F6500CC208227F011278824002C208BD
:01797F0022E5
:107ADC007F021278825007C209C20EC20C227F02AA
:087AEC001278824002C2092257
:107AF4007F031278825007C209C20EC20C227F0390
:087B04001278824002C20E2239
:107B0C007F041278825007C209C20EC20C227F0475
:087B1C001278824002C20C2223
:1069E6000500050105030507050F051F051E051C06
:1069F600051805100201040E040A03060101040B22
:106A06000304040F020304010302040D0200020240
:106A16000300040904040305030701000303040734
:106A2600030104060402040C0516051500000615EC
:0E6A3600062A060C06380633061E0612061740
:10529900203737900640E004F519D3648094815093
:1052A90003025373D3E5196480948F400375190F72
:1052B90090063DE0FF123E6090063EE0F518E4F5E9
:1052C9001ED237C264C257C24A22304A60306416BD
:1052D900152EE52ED394004003025373C2CAC2644B
:1052E900D25785182E2230570E152EE52ED394004D
:1052F9005078C264C25722AF1C151CEF700BC24A0A
:10530900E51825E0F52ED25722E51D30E005851870
:105319002E8008E51875F003A4F52EAF1D7801EF6E
:1053290008800103D8FDF51DD264D2CA22D5190817
:10533900C237E4F53DC25822051E7440251EF58288
:10534900E43406F583E025E024E6F582E43469F5E2
:1053590083E493540FF51C740193F51D700AD25719
:0A536900E51825E025E0F52ED24AF4
:015373002217
:105F990020371A90063DE0FF123E6090063EE0F57C
:105FA9001AE4F51ED237C264C257C24A22304A598E
:105FB900306413152EE52ED39400506BC2CAC26407
:105FC900D257851A2E2230570E152EE52ED394005E
:105FD9005055C264C25722AF1C151CEF7007C24A44
:105FE900C237F53D22E51D30E005851A2E8008E50A
:105FF9001A75F003A4F52EAF1D7801EF088001038F
:10600900D8FDF51DD264D2CA22E53F25E024E6F584
:1060190082E43469F583E493FA740193FBEA540F3B
:07602900F51CEBF51DD24A46
:01603000224D
:107BA100C3EF648094A15008EF25E025E0F52E2273
:047BB100E4F52E22A7
:10752700BF010790063E7418F022BF020790063E7F
:107537007412F022BF030590063E8014BF04079023
:10754700063E740BF02290063EBF05047409F02234
:04755700740CF0229E
:103E6000EF14B420004003023FB3903E7875F00396
:103E7000A4C58325F0C58373023ED8023EDF023E0F
:103E8000E6023EED023EF4023EFB023F02023F0923
:103E9000023F10023F17023F1E023F25023F2C0245
:103EA0003F33023F3A023F41023F48023F4F023F49
:103EB00056023F5D023F64023F6B023F72023F7950
:103EC000023F80023F87023F8E023F95023F9702EA
:103ED0003F9E023FA5023FAC75CB8E75CAC62275C8
:103EE000CB9575CA772275CB9B75CA692275CBA015
:103EF00075CABA2275CBA675CA332275CBAB75CA03
:103F0000632275CBB075CA022275CBB475CAA322E1
:103F100075CBB875CAFA2275CBBC75CAD82275CBD9
:103F2000C075CAA82275CBC475CA362275CBC775B1
:103F3000CA862275CBCA75CABC2275CBCD75CAB4E8
:103F40002275CBD075CA762275CBD375CA3022754F
:103F5000CBD575CAB22275CBD875CA132275CBDA08
:103F600075CA522275CBDC75CA7D2275CBDD75CA48
:103F70006E2275CBE075CA542275CBE275CA1B223E
:103F800075CBE375CAC32275CBE575CA5E2275CBC6
:103F9000E675CADA22801C75CBE875CA902275CB0B
:103FA000EA75CAD92275CBEC75CA092275CBED75B5
:0A3FB000CA292275CBE875CA412228
:10724900EFC39400403FEF9408503AE4FEEF75F025
:1072590008A42430F582E43400F583E5822EF58212
:10726900E43583F583E0FCED75F008A424E8F582A4
:10727900E4341AF583E5822EF582E43583F583EC4F
:05728900F00EBE08C874
:01728E0022DD
:1060C7008F5BE55B6405701D200A0DD20A7FF47EA5
:1060D70001127A8DC20A8074C20A7FF47E01127A95
:1060E7008DD20A8067E55B6406701D200B0DD20B0D
:1060F7007FF47E01127A8DC20B800BC20B7FF47E78
:1061070001127A8DD20B8044E55B6407701D200F66
:106117000DD20F7FF47E01127A8DC20F800BC20F52
:106127007FF47E01127A8DD20F8021E55B640870BF
:1061370022200D0DD20D7FF47E01127A8DC20D80C3
:106147000BC20D7FF47E01127A8DD20D7FF47E0192
:04615700127A8D2209
:104EC200A233B330B401B350357D017F081262734F
:104ED2005027A233B35010A2B4B3500B900652E045
:104EE200FF7C077D30800F30330F30B40C900653B7
:104EF200E0FF7C077D50127357A2B4B39233A23401
:104F0200B330B501B350357D027F0812627350276A
:104F1200A234B35010A2B5B3500B900654E0FF7CFC
:104F2200077D70800F30340F30B50C900655E0FFCE
:104F32007C077D90127357A2B5B39234A235B33079
:104F4200B701B350357D037F081262735027A23533
:104F5200B35010A2B7B3500B900656E0FF7C077D0A
:104F6200B0800F30350F30B70C900657E0FF7C074A
:104F72007DD0127357A2B7B39235A236B330B601C1
:104F8200B350357D047F081262735027A236B350A6
:104F920010A2B6B3500B900658E0FF7C077DF0805C
:104FA2000F30360F30B60C900659E0FF7C087D10AA
:094FB200127357A2B6B392362225
:1076E200900027E0FF30E404D20A8002C20AEF30A1
:1076F200E504D20B8002C20BEF30E604D20F800207
:0B770200C20FEF30E703D20D22C20DD2
:01770D002259
:1074870090063CE0FF602E20370F6029123E60D245
:10749700CAD237D264752E1422E52ED39400400346
:1074A700152E22206408D2CA752E14D26422C2CAAD
:0674B700752E7DC2642267
:1074BD002037127F1C123E60D2CAD237D264752E8D
:1074CD0064751B3C22E52ED394004003152E22AF8C
:1074DD001B151BD3EF648094804004752E6422C26B
:0474ED0037E4F53D4E
:0174F1002278
:104FBB0020371C754006E53E75F008A424E8F58201
:104FCB00E4341AF583E06003D23722E4F53D22E5A1
:104FDB002ED394004003152E22C2CA1540E540146F
:104FEB00700302507614606F14604014602E1460CE
:104FFB00030250AAE53E75F008A424E8F582E434D8
:10500B001AF583E0FF7003F53D22123E60E53E7515
:10501B00F008A424E9F582E4341A8079E53E75F0B2
:10502B0008A424EAF582E4341A80397408441B700E
:10503B0003F53D22E53E75F008A424EBF582E4343C
:10504B001AF583E0FF123E60E53E75F008A424ECF0
:10505B00F582E4341A803EE53E75F008A424EDF5A4
:10506B0082E4341AF583E0FF027BA17420441B70A9
:10507B0003F53D22E53E75F008A424EEF582E434F9
:10508B001AF583E0FF123E60E53E75F008A424EFAD
:10509B00F582E4341AF583E0FF127BA1D2CA22E435
:0750AB00F53DC2CAC2372225
:10755B00E53D14601C14601C14601C14601F146047
:10756B001F2405701EC2CAC237C264C257E4F5405D
:10757B0022024FBB027487125299D258220274BD59
:04758B00125F9922D0
:10768800E52365437004E5226542601F8522428533
:107698002343C2A4D2A5C2A6C2A700AF23127B3A35
:0D76A800E522FF127B3A00D2A7D322C322B5
:107A5500E52465446014852444D2A4D2A5C2A6C2F7
:0C7A6500A7AF24127B3AD2A7D322C32281
:107A7100E521653C601485213CD2A4C2A5C2A6C201
:0C7A8100A7AF21127B3AD2A7D322C32268
:10422100E4F54CF54D754E1E754FFF854D82854C5D
:1042310083E0F5506350FFE550F0E06550600312F4
:104241007C316350FF854D82854C83E550F0E065FC
:10425100506003127C31054DE54D7002054CE54F70
:10426100154F7002154ED3E54F9400E54E94005062
:10427100BAE4F54CF54DF54EF54FE54D254FF58278
:10428100E54C354EF583E4F0054FE54F7002054EE0
:10429100B4FFE7E54EB41EE275985A758921758819
:1042A10045758845758DE775878075C90275331B1E
:1042B10075341075351B75366075371B7538B075DB
:1042C100391C753A0075B701D2A9D2A8D2AA9006B5
:1042D10000E0FFA3E0901CE0CFF0A3EFF090060216
:1042E100E0FFA3E0901CE2CFF0A3EFF0900604E022
:1042F100FFA3E0901CE4CFF0A3EFF0900606E0FFEF
:10430100A3E0901CE6CFF0A3EFF0901CFA7417F035
:10431100A37499F0901CFC7417F0A37499F0901C8D
:10432100FE7417F0A37499F0901D007417F0A37434
:0943310099F0D291D2AF127790FD
:01433A002260
:027C310080FED3
:1075F600C2AFC284D285BF060AC286E580A2E192E6
:107606006B8018BF070AC286E580A2E2926B800BE8
:10761600BF0808C286E580A2E3926BD286D2AFA2EB
:017626006BF8
:017627002240
:10627300BF0107900020E0FE8048BF020790002185
:10628300E0FE803EBF0307900022E0FE8034BF049F
:1062930007900023E0FE802ABF0507900024E0FE5C
:1062A3008020BF0607900025E0FE8016BF070790F9
:1062B3000026E0FE800CBF0807900027E0FE800266
:1062C300E4FEBD0103EE1322BD0204EEA2E122BDF2
:1062D3000304EEA2E222BD0404EEA2E322BD050400
:1062E300EEA2E422BD0604EEA2E522BD0704EEA25F
:0762F300E622BD0802EE33B4
:0162FA002281
:0250B2008F4D20
:1050B4009000B0E0F54EE54D64017037E54E2402F2
:1050C400FFE433FE7868E66F7001EE60030251A7D7
:1050D4007410254EF582E4341BAF82F5508F51D203
:1050E4006B7F01125A69127A1B12385DC26B7F0101
:1050F4000251A4E54D64027037E54E2402FFE43307
:10510400FE7869E66F7001EE60030251A7746025B2
:105114004EF582E4341BAF82F5508F51D26B7F027F
:10512400125A69127A1B12385DC26B7F020251A4B3
:10513400E54D64037033E54E2402FFE433FE786AE0
:10514400E66F7001EE705C74B0254EF582E4341B9A
:10515400AF82F5508F51D26B7F03125A69127A1BBA
:1051640012385DC26B7F038037E54D64047034E50B
:105174004E2402FFE433FE786BE66F7001EE702379
:105184007400254EF582E4341CAF82F5508F51D261
:105194006B7F04125A69127A1B12385DC26B7F044A
:0351A400125A6933
:0151A70022E5
:04385D008F4FE4FDA8
:023861008D5781
:1038630075F020EFA42460F582E5F03403AF82F510
:103873005A8F5BF583E0F558D3940050030239E97E
:10388300E558941040030239E9E557704C7FF47E04
:1038930001127A8DE55825E0F558755901E558244C
:1038A30001FFE433FEC3E5599FEE6480F87480980A
:1038B30040030239E9E55B2559F582E4355AF5837E
:1038C300E0FFE55B2559F582E4355AF583A3E0FD76
:1038D3001277660559055980C4E5576401707AC2A9
:1038E3002B7FF47E01127A8DE55825E0F558755942
:1038F30001E5582401FFE433FEC3E5599FEE6480DC
:10390300F874809840030239E9E55B2559F582E4B0
:10391300355AF583E0FFE55B2559F582E4355AF521
:1039230083A3E0FD12776690001FE0FF30E00630CE
:103933004903C22022EF30E106304D03C22122EFBA
:1039430030E206305103C22222EF30E30630540343
:10395300C22322055905598098E557640260030282
:1039630039E9C22BC22CC22DC22E7FF47E01127AFA
:103973008DE55825E0F558755901E5582401FFE414
:1039830033FEC3E5599FEE6480F87480985057E581
:103993005B2559F582E4355AF583E0FFE55B25594C
:1039A300F582E4355AF583A3E0FD12776690001F94
:1039B300E030E005303902802290001FE030E1055D
:1039C300303A02801690001FE030E205303B02805F
:1039D3000A90001FE030E308303C05C2200272D495
:0639E3000559055980940E
:0139E90022BB
:024678008F4D64
:10467A00C2679000A8E0FFE54DB401167868E6FE2F
:10468A00D39F400EEE9FF55074102FF582E4341B31
:10469A00804FE54DB402167869E6FED39F400EEED0
:1046AA009FF55074602FF582E4341B8034E54DB4D5
:1046BA000316786AE6FED39F400EEE9FF55074B05B
:1046CA002FF582E4341B8019E54DB4041C786BE69F
:1046DA00FED39F4014EE9FF55074002FF582E43408
:1046EA001CAF82F5518F52D267206703024788D2E6
:1046FA006BAF4D125A697FF47E01127A8D7D207F4D
:10470A00051277667D1A7F081277667FC87E0012C7
:10471A007A8DE4F54EE54EC39550505B0552E5524D
:10472A00AE517002055114F5828E83E0F54F603662
:10473A0024F5601414601714601A14601D146020A4
:10474A0024057028E4FD80277D5F7F0780227D5E37
:10475A007F06801C7D0A7F0280167D327F028010D0
:10476A007D467F02800A7D0A7F038004AD4FE4FF05
:0E477A00127766054E809EC26BAF4D125A69D3
:01478800220E
:1077E30030290F900671E0FF7C0B7D10127357B2A6
:1077F3002922202912900670E0FF7C0A7DF0127383
:0878030057B229E4786CF6226B
:106031007D3F7F091277667D507F08127766900059
:106041000EE493FDE4FF1277667D5B7F06127766AF
:1060510090000FE493FDE4FF127766900010E49343
:10606100FDE4FF127766900011E49324BFB40800A9
:10607100505390608175F003A4C58325F0C58373E7
:1060810002609902609D0260A10260A70260AD02F8
:1060910060B30260B90260BF7D0A80067D32800272
:1060A1007D467F02801C7D0A7F0380167D287F0349
:1060B10080107D467F03800A7D0A7F0480047D284D
:0660C1007F041277662245
:10785B008F53D26B125A697D4B7F021277667D0470
:10786B00E4FF1277667D387F04127766126031C2AF
:07787B006BAF53125A6922A2
:0B7A1B00855182855083E0FFA3E0FD51
:107A2600BF0A02E4FFBD0A02E4FDEF75F00AA42DC9
:027A3600FF222D
:10537400C267D208D2207FF47E01127A8D7D2E7FFF
:10538400031277667D607F02127766C208C220121C
:1053940033467F081275F640030254403049F01238
:1053A40033462049FA7868E6640770427E007F70CD
:1053B40075331B7534108F828E837407F07D01E57D
:1053C400342DF582E43533F583E58224FFF582E557
:1053D4008334FFF583E0F9EF2DF582E43EF583E9AC
:1053E400F00DBD08DAD2677F647E00127A8D7F08E3
:1053F4001275F65047206703025376D208D2207FF5
:10540400F47E01127A8D7D607F021277667D327F91
:10541400061277667D1E7F05127766C208C2207C5D
:10542400007D707B087F787E001267E97F08127523
:10543400F650097F327E00127A8D80F0126D607F03
:06544400647E00127A8D67
:01544A00223F
:1077BA00E4F53DC258C258F532302F05C22FC23FF8
:1077CA0022303005C230C24122303105C231C243B3
:0977DA0022303204C232C2452201
:10433B007580FFC286E580540FFFC285E580C454AB
:10434B00F04FF520D2867D027F0112627340107D03
:10435B00037F011262734007300004D23980287D3D
:10436B00027F01126273500A300007300104D23908
:10437B0080157D037F01126273500A200003300108
:10438B0004D2398002C2397D027F0212627340105F
:10439B007D037F021262734007300204D23A8028F9
:1043AB007D027F02126273500A300207300304D27F
:1043BB003A80157D037F02126273500A200203308C
:1043CB000304D23A8002C23A7D027F031262734029
:1043DB00107D037F031262734007300404D23B80CD
:1043EB00287D027F03126273500A300407300504E4
:1043FB00D23B80157D037F03126273500A200403A6
:10440B00300504D23B8002C23B7D027F04126273F3
:10441B00400F7D037F041262734006300603D23CCB
:10442B00227D027F041262735009300606300703A7
:10443B00D23C227D037F04126273500920060330A5
:07444B000703D23C22C23C32
:014452002247
:10334600202B6EC25A20391C205019901CFAE070AE
:1033560002A3E0700B7D067F011262735002D24712
:10336600C249804D30392130501E901CE0E0700279
:10337600A3E0700B7D087F011262735002D23D30CC
:103386006502D25BD2498029303908205005126D7A
:1033960060801E20391B305018D25AC249C250C212
:1033A60014C210C21CC21812795F7868E66002D295
:1033B6005B202C71203A1C205319901CFCE07002F3
:1033C600A3E0700B7D067F021262735002D24BC2DD
:1033D6004D8052303A28305325901CE2E07002A30B
:1033E600E070127D087F0212627350097F02127824
:1033F600825002D23E306602D25BD24D8027303AEE
:1034060008205305126DB4801C203A19305316C299
:103416004DC253C215C211C21DC219127ADC786997
:10342600E66002D25C202D71203B1C205519901CB1
:10343600FEE07002A3E0700B7D067F0312627350FC
:1034460002D24EC2518052303B28305525901CE4A2
:10345600E07002A3E070127D087F031262735009C8
:103466007F031278825002D240302802D25BD251BA
:103476008027303B08205505126E08801C203B191A
:10348600305516C251C255C216C212C21EC21A12F7
:103496007AF4786AE66002D25D202E6D203C1B200D
:1034A6005618901D00E07002A3E0700B7D067F04A5
:1034B6001262735002D252C25422303C2730562434
:1034C600901CE6E07002A3E070127D087F04126291
:1034D6007350097F041278825002D242302A02D2F7
:1034E6005BD25422303C06205603026E5C203C1907
:1034F600305616C254C256C217C213C21FC21B127E
:0A3506007B0C786BE66002D26022B5
:047C2A001251A82229
:1051A80090001FE0540FFFBF010B304906203D035C
:1051B80002526FC322EF64037014304906203D0386
:1051C80002526F304D06203E0302527AC322EF642A
:1051D800057014304906203D0302526F30510620F5
:1051E8004003025285C322EF640970133049052039
:1051F8003D028073305406204203025290C322EFCE
:105208006407701A304905203D02805B304D052047
:105218003E02805E3051052040028061C322EF6467
:105228000B701A304905203D02803C304D05203E68
:1052380002803F305405204202804DC322EF640DA6
:10524800701A304905203D02801D3051052040026A
:10525800802B305405204202802EC322EF640F7049
:105268002E304908203D05753E01D322304D0820D7
:105278003E05753E02D322305108204005753E0395
:10528800D322305408204205753E04D322C322C3DA
:0152980022F3
:10788200BF010690001FE01322BF020790001FE015
:10789200A2E122BF030790001FE0A2E222BF04067A
:0778A20090001FE0A2E322A9
:106D60007868E6602275331B753410E4FFE5342F34
:106D7000F582E43533F583E4F00FBF50F075331B33
:106D8000753410E47868F6900600E0FFA3E0901CEC
:106D9000E0CFF0A3EFF0900608E0FFA3E0901CFA2C
:106DA000CFF0A3EFF0C246C247C25FC23DC265C288
:036DB0003FD2507F
:016DB30022BD
:106DB4007869E6602275351B753660E4FFE5362F89
:106DC400F582E43535F583E4F00FBF50F075351BDB
:106DD400753660E47869F6900602E0FFA3E0901C43
:106DE400E2CFF0A3EFF090060AE0FFA3E0901CFCD2
:106DF400CFF0A3EFF0C248C24BC261C23EC266C22A
:036E040041D25325
:016E07002268
:106E0800786AE6602275371B7538B0E4FFE5382FDD
:106E1800F582E43537F583E4F00FBF50F075371B82
:106E28007538B0E4786AF6900604E0FFA3E0901C99
:106E3800E4CFF0A3EFF090060CE0FFA3E0901CFE77
:106E4800CFF0A3EFF0C24CC24EC262C240C228C209
:036E580043D255CD
:016E5B002214
:106E5C00786BE6602275391C753A00E4FFE53A2F31
:106E6C00F582E43539F583E4F00FBF50F075391C29
:106E7C00753A00E4786BF6900606E0FFA3E0901CF0
:106E8C00E6CFF0A3EFF090060EE0FFA3E0901D001C
:106E9C00CFF0A3EFF0C24FC252C263C242C22AC2A9
:036EAC0045D25676
:016EAF0022C0
:1059B400C208C209C20EC20C127A71C267D25EE476
:1059C400F53D7FE87E03127A8DC298C2AF75567F8B
:1059D400755596755498755300785374FF125996FB
:1059E400E4FBFAF9F8C3125983504430983E12008C
:1059F40006127BECEF14601824F0602624C1600BBF
:105A040024F670287F06127C1A80211271B9801C3A
:105A14007F06127C1A12758F1276E2127091D26789
:105A2400800A7F06127C1A126778D2673067AAE46C
:105A3400786CF6D26B7F01125A697F01126C0A7D71
:105A4400467F021277667D1E7F071277667D147F7C
:105A5400081277667D327F03127766C26B7F01126C
:045A64005A69C25E5B
:015A6800221B
:10677800756701756500756620E4F5577F02127C20
:106788001AE5672402F559AF67127C1AE4F558E553
:10679800662558F582E43565F583E0FF127C1AE535
:1067A800662558F582E43565F583E02559F55905E0
:1067B80058E558C3948040D7AF59127C1A7F03120A
:1067C8007C1A127C22EF64156016056774802566B2
:1067D800F566E43565F5650557E557C39435409C7E
:0167E800228E
:10758F00756701756500756620E4F5571276B5507D
:10759F00077F06127C1A80057F15027C1A05677417
:1075AF00802566F566E43565F5650557E557C3949F
:0375BF003540D97B
:0175C20022A6
:1076B500E4F558127C2274502558F582E4341CF503
:1076C50083EFF00558E558C3948440E7127B50904A
:0C76D5001CD2E0B50705127980D322C357
:0176E1002286
:10798000E4FF74522FF582E4341CF583E0FEE566D3
:0F7990002FF582E43565F583EEF0000FBF80E33D
:01799F0022C5
:107B5000E4FFFE74502EF582E4341CF583E02FFF21
:047B60000EBE82EFE4
:017B640022FE
:1071B900E4F557F55D755CE0755B93755A04F5590F
:1071C900785974FF125996E4FBFAF9F8C3125983F6
:1071D90050253098EB1200068F58E5586404601763
:1071E900AF5D055D74502FF582E4341CF583E558D5
:0771F900F02557F55780C98E
:01720000226B
:04000600AF99C29854
:01000A0022D3
:087C1A003099FDC2998F9922F7
:077C22003098FDAF99C298F4
:017C29002238
:105BD100070102030405060707070605040302017E
:105BE10003010A0A03020A0A03030A0A03040A0A4E
:105BF100030307050303020503070A0A04024B0016
:105C0100040438072E03024B0004043802055F0028
:105C11000302055F000402055F000502055F00063F
:105C210002055F000702055F000802055F00090227
:105C3100055F000A02055F000B02055F000C02050B
:105C41005F000D02055F000E02055F000F02055F98
:105C5100001002055F001102055F001204072E0803
:105C6100260640033204072E082606400253080C7C
:075C71000A1D040000241BC2
:10001600C2AF9000207491F09000217481F090009E
:1000260022F0900023F09000247403F090002574D1
:10003600BFF09000267418F0900027740FF090001F
:10004600307409F0A37403F0E4A3F0A37410F0A3D2
:100056007403F0E4A3F0A37415F0A37403F0A3747F
:1000660015F0A37403F0E4A3F0A37410F0A37403D3
:10007600F0E4A3F0A37409F0A37403F0A37415F0DD
:10008600A37403F0A314F0A3741AF0A37403F0E4AA
:10009600A3F0A3F0A3F0A3741AF0A37403F0A314BF
:1000A600F0A37415F0A37403F0E4A3F0A3F0A3F097
:1000B6007E5B7FE17C007D807B041273167E5B7F16
:1000C600E57C007D887B041273167E5B7FE97C00ED
:1000D6007D907B041273167E5B7FED7C007D987BA2
:1000E600041273167E5B7FF57C007DA07B04127381
:1000F600167E5B7FF17C007DA87B041273167E5B07
:100106007FF97C007DB07B041273167E5B7FD17C09
:10011600007D707B081273167E5B7FD97C007D782C
:100126007B081273167E5B7FFD7C037D807B091244
:1001360073167E5C7F067C037DA07B071273167E9A
:100146005C7F0D7C037DC07B051273167E5C7F127F
:100156007C037DE07B051273167E5C7F177C047D35
:10016600007B051273167E5C7F1C7C047D207B055C
:100176001273167E5C7F217C047D407B051273160C
:100186007E5C7F267C047D607B051273167E5C7F19
:100196002B7C047D807B051273167E5C7F307C048D
:1001A6007DA07B051273167E5C7F357C047DC07B4B
:1001B600051273167E5C7F3A7C047DE07B05127324
:1001C600167E5C7F3F7C057D007B051273167E5C88
:1001D6007F447C057D207B051273167E5C7F497CFF
:1001E600057D407B051273167E5C7F4E7C057D6027
:1001F6007B051273167E5C7F537C057D807B051222
:1002060073167E5C7F587C057DA07B051273167E77
:100216005C7F5D7C057DC07B091273167E5C7F6604
:100226007C057DE07B09127316900600E4F0A3744A
:10023600B4F0900602E4F0A374B4F0900604E4F07F
:10024600A374B4F0900606E4F0A374B4F090061814
:100256007401F0A374E0F090061AE4F0A37478F049
:1002660090061EE4F0A3743CF09006087402F0A316
:100276007458F090060A7402F0A37458F090060CB5
:100286007402F0A37458F090060E7402F0A374582A
:10029600F09006107401F0A3742CF090061274020C
:1002A600F0A37458F09006147403F0A37484F090CD
:1002B60006167404F0A374B0F07407900620F0A339
:1002C600F0900622F0A3F090061C7402F0A3745876
:1002D600F0900630740AF09006317428F0900633D8
:1002E600740AF0900634F09006327405F07E5C7F56
:1002F6006F7C067D407B0912731690063D7417F0DD
:1003060090063E740CF090063C7419F0E490063F9B
:10031600F090063B740CF09006527401F090073092
:100326007469F0A37411F09006537401F0900750AD
:100336007469F0A37410F09006547401F09007707D
:100346007469F0A37421F09006557401F09007903B
:100356007469F0A37420F09006567401F09007B00B
:100366007469F0A37431F09006577401F09007D0C9
:100376007469F0A37430F09006587401F09007F099
:100386007469F0A37441F09006597401F090081056
:100396007469F0A37440F090065A7401F090083026
:1003A6007462F0A37411F0A37432F0A37401F0A385
:1003B6007450F0A37410F090065B7401F09008502E
:1003C6007461F0A37420F0A37462F0A37411F0A317
:1003D6007432F0A37402F0A37450F0A37410F0907A
:1003E600065C7401F09008707451F0A37411F0A3C8
:1003F6007433F0A3E4F0A37451F0A37410F09006E4
:100406005D7401F09008907462F0A37411F0A37407
:1004160030F0A37402F0A37462F0A37410F0900697
:100426005E7401F09008B07451F0A37411F0A374D7
:1004360041F0A37410F0A37451F0A37410F0900669
:100446005F7401F09008D07451F0A37411F0A37496
:1004560034F0A37414F0A37451F0A37410F0900652
:10046600607401F09008F07451F0A37411F0A37455
:1004760034F0A37418F0A37451F0A37410F090062E
:10048600617401F09009107451F0A37411F0A37413
:1004960034F0A37428F0A37451F0A37410F09006FE
:1004A600627401F09009307462F0A37411F0A374C1
:1004B60030F0A37403F0A37462F0A37410F09006F6
:1004C600637401F09009507462F0A37411F0A37480
:1004D60030F0A37404F0A37462F0A37410F09006D5
:1004E600647401F09009707462F0A37411F0A3743F
:1004F60060F0A37401F0A37495F0A3743DF0A374A7
:1005060090F0A37401F0A37498F0A37426F0A3747A
:1005160096F0A37440F0A37462F0A37410F0A37471
:1005260061F0A37470F09006657401F09009907400
:1005360062F0A37411F0A37460F0A37401F0A374C5
:1005460095F0A3743DF0A37490F0A37401F0A37426
:1005560096F0A37438F0A37462F0A37410F09006BA
:10056600667401F09009B07462F0A37411F0A3747C
:1005760060F0A37401F0A37495F0A3743DF0A37426
:1005860090F0A37402F0A37498F0A37426F0A374F9
:1005960096F0A37440F0A37462F0A37410F0A374F1
:1005A60061F0A37470F09006677401F09009D0743E
:1005B60062F0A37411F0A37460F0A37401F0A37445
:1005C60095F0A3743DF0A37490F0A37402F0A374A5
:1005D60096F0A37438F0A37462F0A37410F090063A
:1005E600687401F09009F07462F0A37411F0A374BA
:1005F60060F0A37401F0A37495F0A3743DF0A374A6
:1006060090F0A37403F0A37498F0A37426F0A37477
:1006160096F0A37440F0A37462F0A37410F0A37470
:1006260061F0A37470F09006697401F0900A10747A
:1006360062F0A37411F0A37460F0A37401F0A374C4
:1006460095F0A3743DF0A37490F0A37403F0A37423
:1006560096F0A37438F0A37462F0A37410F09006B9
:100666006A7401F0900A307462F0A37411F0A374F6
:1006760060F0A37401F0A37495F0A3743DF0A37425
:1006860090F0A37404F0A37498F0A37426F0A374F6
:1006960096F0A37440F0A37462F0A37410F0A374F0
:1006A60061F0A37470F090066B7401F0900A5074B8
:1006B60062F0A37411F0A37460F0A37401F0A37444
:1006C60095F0A3743DF0A37490F0A37404F0A374A2
:1006D60096F0A37438F0A37462F0A37410F0900639
:1006E6006C7401F0900A707462F0A37411F0A37434
:1006F60060F0A37401F0A37430F0A37405F0A37442
:1007060062F0A37410F090066D7401F0900A907474
:1007160062F0A37421F0A37460F0A37401F0A374D3
:1007260030F0A37406F0A37462F0A37420F0900670
:100736006E7401F0900AB07462F0A37431F0A37481
:1007460060F0A37401F0A37430F0A37407F0A374EF
:1007560062F0A37430F090066F7401F0900AD074C2
:1007660062F0A37441F0A37460F0A37401F0A37463
:1007760030F0A37408F0A37462F0A37440F09006FE
:10078600707401F0900AF07464F0A37411F0A3740D
:1007960096F0A37432F0A37495F0A3741EF0A374BC
:1007A60098F0A3744BF0A37464F0A37410F0900651
:1007B600717401F0900B107464F0A37411F0A374BB
:1007C60096F0A37432F0A37495F0A3741EF0A3748C
:1007D60093F0A37418F0A37464F0A37410F0900659
:1007E600737401F0900B507462F0A37411F0A3744B
:1007F60060F0A37401F0A37495F0A3743DF0A374A4
:1008060090F0A37402F0A37497F0A37426F0A37477
:1008160093F0A37418F0A37462F0A37410F0A37499
:1008260070F0A37410F09006747401F0900B70745D
:1008360062F0A37411F0A37460F0A37401F0A374C2
:1008460095F0A3743DF0A37490F0A37403F0A37421
:1008560097F0A37426F0A37493F0A37418F0A3740E
:1008660062F0A37410F0A37470F0A37420F09006E5
:10087600757401F0900B907462F0A37411F0A37478
:1008860060F0A37401F0A37495F0A3743DF0A37413
:1008960090F0A37404F0A37497F0A37426F0A374E5
:1008A60093F0A37418F0A37462F0A37410F0A37409
:1008B60070F0A37430F09006817401F0900D1074FE
:1008C60062F0A37411F0A37460F0A37401F0A37432
:1008D60092F0A3744BF0A37490F0A37404F0A37485
:1008E60094F0A37438F07499A3F0A3F0A37460F0A5
:1008F600A37401F0A37462F0A37410F01222F8122C
:100906007091D26B7F01125A697D2F7F071277662D
:100916007D0C7F031277667D327F061277667D1E19
:100926007F0512776690001F7401F0FD7F1F7E0021
:0B093600127397C26B7F01125A6922F6
:1022F8009001007402F0A3740DF0A37402F090062C
:10230800A014F09010F07464F0A37411F0A3749703
:10231800F0A3742EF0A37495F0A3743DF0A3749009
:10232800F0A37402F0A37496F0A37438F0A3746455
:10233800F0A37410F0A37470F0A37411F090010866
:102348007402F0A3740EF0A37402F09006A114F0C6
:102358009011107461F0A37410F0A37464F0A37466
:1023680011F0A37497F0A3742EF0A37495F0A374DE
:102378003DF0A37490F0A37402F0A37496F0A374D4
:1023880036F0A37464F0A37410F0A37470F0A3740F
:1023980010F09001107402F0A3740DF0A37403F010
:1023A8009006A27401F09011307464F0A37411F0D7
:1023B800A37497F0A3742EF0A37495F0A3743DF062
:1023C800A37490F0A37403F0A37496F0A37438F088
:1023D800A37464F0A37410F0A37470F0A37421F0D4
:1023E8009001187402F0A3740EF0A37403F0900621
:1023F800A37401F09011507461F0A37410F0A374E9
:1024080064F0A37411F0A37497F0A3742EF0A3746E
:1024180095F0A3743DF0A37490F0A37403F0A37433
:1024280096F0A37436F0A37464F0A37410F0A37448
:1024380070F0A37420F09001207402F0A3740DF0E2
:10244800A37404F09006A47401F09011707464F001
:10245800A37411F0A37497F0A3742EF0A37495F0ED
:10246800A3743DF0A37490F0A37404F0A37496F0E1
:10247800A37438F0A37464F0A37410F0A37470F01C
:10248800A37431F09001287402F0A3740EF0A374C1
:1024980004F09006A57401F09011907461F0A37493
:1024A80010F0A37464F0A37411F0A37497F0A374EC
:1024B8002EF0A37495F0A3743DF0A37490F0A37468
:1024C80004F0A37496F0A37436F0A37464F0A374B4
:1024D80010F0A37470F0A37430F09001307403F01E
:1024E800A3740DF0A37402F0A304F09006A674017F
:1024F800F09011B07464F0A37411F0A37497F0A372
:10250800742EF0A37495F0A3743DF0A37490F0A317
:102518007402F0A37490F0A37403F0A37496F0A36C
:102528007438F0A37464F0A37410F0A37470F0A36B
:102538007441F09001387403F0A3740EF0A3740290
:10254800F0A304F09006A77401F09011D07461F024
:10255800A37410F0A37464F0A37411F0A37497F03B
:10256800A3742EF0A37495F0A3743DF0A37490F0B7
:10257800A37402F0A37490F0A37403F0A37496F00C
:10258800A37436F0A37464F0A37410F0A37470F00D
:10259800A37440F09001407404F0A3740DF0A37488
:1025A80002F0A304F0A304F09006A87401F09011BF
:1025B800F07464F0A37411F0A37497F0A3742EF070
:1025C800A37495F0A3743DF0A37490F0A37402F083
:1025D800A37490F0A37403F0A37490F0A37404F0B0
:1025E800A37496F0A37438F0A37464F0A37410F085
:1025F800A37470F0A37441F0A37470F0A37451F045
:102608009001487404F0A3740EF0A37402F0A304BC
:10261800F0A304F09006A97401F09012107461F010
:10262800A37410F0A37464F0A37411F0A37497F06A
:10263800A3742EF0A37495F0A3743DF0A37490F0E6
:10264800A37402F0A37490F0A37403F0A37490F041
:10265800A37404F0A37496F0A37436F0A37464F022
:10266800A37410F0A37470F0A37440F0A37470F016
:05267800A37450F022E4
:0A7316008E4C8F4D8C4E8D4F8B5026
:10732000E4F9C3E5506480F8E96480985028E9FFE7
:107330003395E0FEE54D2FF582E54C3EF583E49371
:10734000FFE9FD3395E0FCE54F2DF582E54E3CF578
:0673500083EFF00980CC80
:017356002214
:107AC200D291C2A4C2A5C2A6C2A7007F05127B3A68
:097AD20000127B2400D2A7D2911E
:017ADB002288
:1079DF00127AC2EF20E0F9D291C2A4C2A5C2A6C208
:0E79EF00A7007F06127B3A0000D2A7D2912299
:1079FD00127AC2EF20E0F9D291C2A4C2A5C2A6C2EA
:0E7A0D00A7007F04127B3A0000D2A7D291227C
:046EB0008E528F531C
:106EB400AE04AF058E568F57D291C2A4C2A5C2A606
:106EC400C2A7007F03127B3AE552FF127B3AAF530D
:106ED400127B3AE4F554F555127B24E5572555F514
:106EE40082E5563554F583EFF00555E555700205F6
:0E6EF40054C39420E554940040DED2A7D291FE
:016F0200226C
:086927008E5D8F5E8C5F8D60B8
:10692F00127AC2EF20E0F91279DF855D63855E642C
:10693F00D291C2A4C2A5C2A6C2A7007F02127B3AFF
:10694F00E55FFF127B3AAF60127B3AE4F561F562C7
:10695F00E5642562F582E5633561F583E0FF127B1F
:10696F003A0562E56270020561C39420E561940007
:07697F0040DE00D2A7D29117
:0169860022EE
:0A67E9008E4C8F4D8C4E8D4F8B505F
:1067F300C2AF1279DF127AC2EF20E0F9854E5285DB
:106803004F53D291C2A4C2A5C2A6C2A7007F02124F
:106813007B3AE54CFF127B3AAF4D127B3AE4F551DC
:10682300AF50EF3395E0FEC3E5519FEE6480F874FB
:1068330080985014E5532551F582E43552F583E0F1
:10684300FF127B3A055180D800D2A7D2911279FD6D
:02685300D2AFC2
:016855002220
:107397008E5B8F5C8D5DC2AF1279DF127AC2EF20F0
:1073A700E0F9D291C2A4C2A5C2A6C2A7007F021269
:1073B7007B3AE55BFF127B3AAF5C127B3AAF5D121B
:0E73C7007B3A0000D2A7D2911279FDD2AF22FC
:0478A9008E4C8F4D25
:1078AD00D291C2A4C2A5C2A6C2A77F03127B3AE59C
:1078BD004CFF127B3AAF4D127B3A127B24D2A7D2EA
:0178CD009129
:0178CE002297
:10720100C2AF754E00754F20755000755120E4F5E1
:107211004CF54DAD4FAC4EAF51AE50126EB0742027
:10722100254FF54FE4354EF54E74202551F551E4C7
:107231003550F550054DE54D7002054CC394D6E52A
:077241004C940040CED2AFD7
:017248002223
:10709100C2AF755B00755C20755900755A20E4F527
:1070A10057F558AD5AAC59AF5CAE5B1269277420E5
:1070B100255AF55AE43559F5597420255CF55CE4F7
:1070C100355BF55B0558E55870020557C394D6E565
:0A70D10057940040CE1279FDD2AFB3
:0170DB002292
:046F55008C4D8D4E84
:106F5900EF6048D22BD22CD22DD22EE4F54F854E9C
:106F690082854D83E0FEA3E04E6028AF4FEF339555
:106F7900E0FEEF25E0FFEE33FEE54E2FF582E54D0D
:106F890012544B926720670B054FC3E54F648094F9
:0B6F99009040CBC22BC22CC22DC22E98
:016FA40022CA
:047357008C4D8D4E7E
:10735B00EF6038E4F54F854E82854D83E0FEA3E068
:10736B004E6028AF4FEF3395E0FEEF25E0FFEE3395
:10737B00FEE54E2FF582E54D12544B926720670BBD
:0B738B00054FC3E54F6480949040CB99
:0173960022D4
:08544B003EF583E0FEA3E0FF43
:04545300AD07AC06EF
:10545700C268780CEF088006A2E0CE13CE13D8F806
:10546700540FF5507808AF05AE04EF088006A2E0A8
:10547700CE13CE13D8F8540FF5517804AF05AE0408
:10548700EF088006A2E0CE13CE13D8F8540FF552DA
:10549700ED540FF553E550607CB4010BAB53AD529F
:1054A700AF5112583E806EE550B4030BAB53AD526B
:1054B700AF51126AA2805EE550B4040BAB53AD52F4
:1054C700AF51126AFD804EE550B4050BAB53AD5298
:1054D700AF51123CEC803EE550B4060BAB53AD52D6
:1054E700AF5112180F802EE550B4070BAB53AD52D6
:1054F700AF51124106801EE550B4080BAB53AD52B5
:10550700AF51126F03800EE550B40909AB53AD528A
:07551700AF511278F4A26805
:01551E00226A
:10583E008F548D558B56E554B40113900020E0FF24
:10584E00126A4A900020EFF0FD7F200258D9E554ED
:10585E00B40211900021126A44900021EFF0FD7FF6
:10586E00210258D9E554B40310900022126A4490D4
:10587E000022EFF0FD7F228052E554B40410900018
:10588E0023126A44900023EFF0FD7F23803DE55400
:10589E00B40510900024126A44900024EFF0FD7FAE
:1058AE00248028E554B40610900025126A44900016
:1058BE0025EFF0FD7F258013E554B40713900026E5
:1058CE00126A44900026EFF0FD7F267E0002739749
:1058DE00E554B40816900027126A44900027EFF0A2
:0C58EE00FD7F277E001273971276E222E5
:066A4400E0FFAB56AD556A
:106A4A00D269AC07BD01047E018033BD02047E0217
:106A5A00802CBD03047E048025BD04047E08801EAC
:106A6A00BD05047E108017BD06047E208010BD0778
:106A7A00047E408009BD08047E808002C269BB0191
:106A8A0005EE4204800BEB7006EEF452048002C25B
:076A9A0069306903AF04221B
:016AA10022D2
:106AA2008F548D558B56E554700BAD56AF55127BF6
:106AB200CCE4FD801EE554B4010BAD56AF55127BFC
:106AC200CC7D01800EE554B4020CAD56AF55127B5D
:106AD200CC7D02023861E554B4030AE55570061212
:106AE20072D4C25822E554B40410AD56AF551267A1
:0B6AF200468F3F753D05E53D70FC221E
:106AFD008F548D558B56E5547036E555B40108E528
:106B0D005614FF7D018026E555B40208E55614FFA5
:106B1D007D028019E555B40308E55614FF7D038009
:106B2D000CE55564047022E55614FF7D040272498C
:106B3D00E554B40114E555D39400400DE555940585
:0A6B4D005007753D01E53D70FC2284
:103CEC008B54EF7017BD0114E5547002C220E554DB
:103CFC0064016003023E58D220023E58EF7017BD9B
:103D0C000214E5547002C221E55464016003023EC2
:103D1C0058D221023E58EF7017BD0314E5547002BF
:103D2C00C222E55464016003023E58D222023E587E
:103D3C00EF7017BD0414E5547002C223E5546401FE
:103D4C006003023E58D223023E58EF701BBD05188B
:103D5C00E5547004C220C221E55464016003023EA4
:103D6C0058D220D221023E58EF701BBD0618E554E4
:103D7C007004C222C223E55464016003023E58D28F
:103D8C0022D223023E58BF0117BD0114E554700224
:103D9C00C224E55464016003023E58D224023E580A
:103DAC00BF0117BD0214E5547002C225E55464012D
:103DBC006003023E58D225023E58BF0116BD0313C4
:103DCC00E5547002C226E55464016003023E58D2E9
:103DDC00268079BF0113BD0410E5547002C227E59B
:103DEC005464017067D2278063BF0117BD0514E5C9
:103DFC00547004C224C225E5546401704FD224D2FD
:103E0C00258049BF0117BD0614E5547004C226C2B3
:103E1C0027E55464017035D226D227802FEF640138
:103E2C00702AED64097025E554B401047F018019F2
:103E3C00E554B402047F028010E554B403047F03FC
:103E4C008007E554B404057F04126C0A7F327E00AF
:043E5C00127A8D2227
:10180F008F548D558B56E5547016AD56AF55127BD0
:10181F00CC901D14EFF0901D14E0D3940050F722DC
:10182F00E554B40117E555B40112E5567002C2082C
:10183F00E55664016003021BB5D20822E554B401DA
:10184F0017E555B40212E5567002C209E556640158
:10185F006003021BB5D20922E554B40117E555B454
:10186F000312E5567002C20EE55664016003021BB7
:10187F00B5D20E22E554B40117E555B40412E5565E
:10188F007002C20CE55664016003021BB5D20C2234
:10189F00E554B4011BE555B40516E5567004C208AE
:1018AF00C209E55664016003021BB5D208D20922B2
:1018BF00E554B40118E555B40613E5567004C20E8D
:1018CF00C20CE55664016003021BB58024E5546425
:1018DF00017023E555B4071EE5567008C208C2090A
:1018EF00C20EC20CE55664016003021BB5D208D2CA
:1018FF0009D20ED20C22E554B4021DE555B40118DD
:10190F00E5567004C208C220E55664016003021B4D
:10191F00B5D208D220021AD5E554B4021DE555B44C
:10192F000218E5567004C209C221E556640160032E
:10193F00021BB5D209D221021A61E554B4021DE58A
:10194F0055B40318E5567004C20EC222E556640161
:10195F006003021BB5D20ED222021A85E554B402DF
:10196F001DE555B40418E5567004C20CC223E556A4
:10197F0064016003021BB5D20CD223021AA8E554EE
:10198F0064027026E55564057020E5567008C2089C
:10199F00C209C220C221E55664016003021BB5D201
:1019AF0008D209D220D221021AD5E554640270263A
:1019BF00E55564067020E5567008C20EC20CC222AF
:1019CF00C223E55664016003021BB5D20ED20CD2BE
:1019DF0022D223021A85E55464027035E555640757
:1019EF00702FE5567010C208C209C20EC20CC22079
:1019FF00C221C222C223E55664016003021BB5D285
:101A0F0008D209D20ED20CD220D221D222D22380D8
:101A1F0065E554B4031DE555B40118E5567004C2CD
:101A2F0008C224E55664016003021BB5D208D22414
:101A3F00021AD5E554B4031FE555B4021AE55670E2
:101A4F0004C209C225E55664016003021BB5D20921
:101A5F00D2257F02021B04E554B4031EE555B403DF
:101A6F0019E5567004C20EC226E5566401600302E2
:101A7F001BB5D20ED2267F03807BE554B4031EE53F
:101A8F0055B40419E5567004C20CC227E55664011B
:101A9F006003021BB5D20CD2277F048058E5546433
:101AAF00037027E55564057021E5567008C208C21A
:101ABF0009C224C225E55664016003021BB5D20892
:101ACF00D209D224D2257F01802BE55464037028DC
:101ADF00E55564067022E5567008C20EC20CC22688
:101AEF00C227E55664016003021BB5D20ED20CD299
:101AFF0026D2277F03026C0AE554B4040AE555B4D5
:101B0F000105AF56026685E554B4040AE555B402E3
:101B1F0005AF560268BFE5546409701EE555B40160
:101B2F0019E5567003C20A22E556B40103D20A2200
:101B3F00E556640270707F058069E5546409701E74
:101B4F00E555B40219E5567003C20B22E556B401F0
:101B5F0003D20B22E5566402704C7F068045E55494
:101B6F006409701EE555B40319E5567003C20F22C0
:101B7F00E556B40103D20F22E556640270287F07A1
:101B8F008021E5546409701EE555B40419E55670BB
:101B9F0003C20D22E556B40103D20D22E556B4025D
:071BAF00057F081260C72248
:104106008F548D558B56E554700FE555700BE5565B
:10411600B40306127044024214E55460030241FCE3
:10412600E555B4010DE556700990001FE054FDF009
:104136008011E555B4010CE556B4010790001FE067
:104146004403F0E555B4020DE556700990001FE0F2
:1041560054FBF08011E555B4020CE556B401079006
:10416600001FE04405F0E555B4030DE556700990CF
:10417600001FE054F7F08011E555B4030CE556B482
:10418600010790001FE04409F0E555B4040DE5561B
:10419600700990001FE054F9F08011E555B4040C45
:1041A600E556B4010790001FE04407F0E555B40555
:1041B6000DE556700990001FE054F3F08011E555A7
:1041C600B4050CE556B4010790001FE0440DF0E578
:1041D60055B4060DE556700990001FE054F1F080C5
:1041E6002DE55564067027E5566401702190001F81
:1041F600E0440FF08018E554B40113E555700FE55F
:10420600567004C2298007E556B40102D2299000EF
:0B4216001FE0FD7F1F7E001273972247
:106F03008F548D558B56E554700C127BC8744F2FDC
:106F1300F58274068020E554B4010C127BC8744FCB
:106F23002FF58274068024E554B40210127BC874D2
:106F33009F2FF58274063EF583E4F022E554B403F3
:106F430010127BC8749F2FF58274063EF58374017B
:026F5300F0222A
:0278F4008F54AF
:1078F600AF057804EF08800123D8FD4BF555E55414
:10790600B40908E555B49903026031AD55AF541278
:02791600776692
:01791800224C
:10668500E545B40109BF0106D220D2088060E54581
:10669500B40109EF7006C220C2088052E545B40274
:1066A50009BF0106D221D2098044E545B40209EFAC
:1066B5007006C221C2098036E545B40309BF01064B
:1066C500D222D20E8028E545B40309EF7006C22216
:1066D500C20E801AE545B40409BF0106D223D20CC7
:1066E500800CE545B40407EF7004C223C20C127A8E
:0A66F50071AF3E126C0A127A5522B2
:1068BF00E545B40108BF0105D224D20822E545B44D
:1068CF000108EF7005C224C20822E545B40208BFD3
:1068DF000105D225D20922E545B40208EF7005C2A1
:1068EF0025C20922E545B40308BF0105D226D20E01
:1068FF0022E545B40308EF7005C226C20E22E54516
:10690F00B40408BF0105D227D20C22E545B4040711
:08691F00EF7004C227C20C2234
:10704400D26BAF45125A69127A7190001FE030E09A
:10705400077D01E4FF12776690001FE030E1077DB1
:1070640002E4FF12776690001FE030E2077D03E43C
:10707400FF12776690001FE030E3077D04E4FF12FF
:0D7084007766C26BAF45125A69127A71220D
:047BC800AD56AF55B2
:0D7BCC00EF75F00AA47C002DFFEC35F0FEF3
:017BD9002289
:020941008F4DD8
:10094300C268E4F53DD25ED26B125A697D4B7F02D9
:100953001277667D04E4FF1277667D387F04127791
:10096300667D607F0212776690061CE0FFA3E0902D
:100973001CE8CFF0A3EFF0C26BAF4D125A69E4F558
:1009830046C208123346E54DB40106A24992678078
:100993001FE54DB40206A24D92678014E54DB403E2
:1009A30006A25192678009E54DB40404A2549267EC
:1009B300901CE8E07002A3E07005D268020F8B3050
:1009C30067C1123346E54DB40106A2499267801F01
:1009D300E54DB40206A24D92678014E54DB40306BB
:1009E300A25192678009E54DB40404A25492672092
:1009F30067D0E54DB4010A754E1B754F10786880BA
:100A03002BE54DB4020A754E1B754F607869801C47
:100A1300E54DB4030A754E1B754FB0786A800DE53A
:100A23004DB4040B754E1C754F00786BE6F550E51D
:100A330050D394005003020F85854F82854E83E087
:100A4300640B6003020F80A3E0FFB40A0AE550B40D
:100A53000205D268020F85EF64017032854F8285EB
:100A63004E83A3A3E064037025E550B40520854FAE
:100A730082854E83A3A3A3E0FFE54F2404F582E41C
:100A8300354EF583E0FDAB4D123FBA020F85854F1E
:100A930082854E83A3E0B40121854F82854E83A3D3
:100AA300A3E0B40415E550D39405400EAB4DAD4F10
:100AB300AC4EAF50123510020F85854F82854E83A1
:100AC300A3E064017032854F82854E83A3A3E06463
:100AD300057025E550B40520854F82854E83A3A379
:100AE300A3E0FFE54F2404F582E4354EF583E0FDF2
:100AF300AB4D126589020F85854F82854E83A3E036
:100B030064017032854F82854E83A3A3E06406702F
:100B130025E550B40520854F82854E83A3A3A3E02A
:100B2300FFE54F2404F582E4354EF583E0FDAB4D3C
:100B3300125C78020F85854F82854E83A3E0B40152
:100B430021854F82854E83A3A3E0B40715E550D3D7
:100B53009405400EAB4DAD4FAC4EAF50124DC60297
:100B63000F85854F82854E83A3E064017032854FE4
:100B730082854E83A3A3E064087025E550B4052065
:100B8300854F82854E83A3A3A3E0FFE54F2404F59D
:100B930082E4354EF583E0FDAB4D126B57020F85B2
:100BA300854F82854E83A3E0B40219854F82854E1B
:100BB30083A3A3E0B4080DE550B40308AF4D127747
:100BC3003A020F85854F82854E83A3E06402702429
:100BD300854F82854E83A3A3E0B40818E550B4047F
:100BE30013854F82854E83A3A3A3E0FFAD4D1278F7
:100BF30033020F85854F82854E83A3E0B4021985A6
:100C03004F82854E83A3A3E0B4090DE550B40308D6
:100C1300AF4D12770E020F85854F82854E83A3E079
:100C230064027024854F82854E83A3A3E0B4091820
:100C3300E550B40413854F82854E83A3A3A3E0FF3D
:100C4300AD4D12780B020F85854F82854E83A3E04D
:100C530064037036854F82854E83A3A3E0640A70D4
:100C630029E55064057023854F82854E83A3A3A392
:100C7300E0FFE54F2404F582E4354EF583E0FD12F1
:100C83007A26AD4D12577F020F85854F82854E839D
:100C9300A3E06403703E854F82854E83A3A3E06483
:100CA300017031E550D39405402A854F82854E83E8
:100CB300A3A3A3E0FFE54F2404F582E4354EF583B7
:100CC300E0FD127A26854D55AB50AD4FAC4E124721
:100CD30089020F85854F82854E83A3E064037036B6
:100CE300854F82854E83A3A3E064027029E5506497
:100CF300057023854F82854E83A3A3A3E0FFE54FB1
:100D03002404F582E4354EF583E0FD127A26AD4DD9
:100D1300127127020F85854F82854E83A3E0B403AA
:100D230019854F82854E83A3A3E0B4030DE550B428
:100D33000308AF4D1273D5020F85854F82854E830D
:100D4300A3E0B40321854F82854E83A3A3E0B404BB
:100D530015E550D39403400EAB4DAD50AF4FAE4E9F
:100D6300125F00020F85854F82854E83A3E0B40393
:100D730019854F82854E83A3A3E0B4050DE550B4D6
:100D83000308AF4D127BDA020F85854F82854E83B0
:100D9300A3E0B4031D854F82854E83A3A3E0B4066D
:100DA30011E550B4050CAD4DAF4FAE4E12744E026B
:100DB3000F85854F82854E83A3E064037024854F9E
:100DC30082854E83A3A3E0B40718E550B4041385CA
:100DD3004F82854E83A3A3A3E0FFAD4D1279A002FA
:100DE3000F85854F82854E83A3E0B4031D854F8213
:100DF300854E83A3A3E0B40811E550B4050CAD4DB3
:100E0300AF4FAE4E127628020F85854F82854E83F3
:100E1300A3E064057022E550B4041D854F82854E1E
:100E230083A3A3E0FF854F82854E83A3A3A3E0FDA5
:100E3300AB4D122D80020F85854F82854E83A3E033
:100E4300B40524E54F2404F582E4354EF583E0B47C
:100E53000B15E550D39405400EAB4DAD50AF4FAEDF
:100E63004E124899020F85854F82854E83A3E06415
:100E7300067022E550B4041D854F82854E83A3A3DB
:100E8300E0FF854F82854E83A3A3A3E0FDAB4D1204
:100E9300267D020F85854F82854E83A3E0B4062409
:100EA300E54F2404F582E4354EF583E0B40B15E5F4
:100EB30050D39405400EAB4DAD50AF4FAE4E1231F3
:100EC3005E020F85854F82854E83A3E064097022FD
:100ED300854F82854E83A3A3E0B40A16E550B4047C
:100EE30011854F82854E83A3A3A3E0FF1270DC021A
:100EF3000F85854F82854E83A3E064097023854F58
:100F030082854E83A3A3E0B40117E550B404128590
:100F13004F82854E83A3A3A3E0FFAD4D1256BB8042
:100F230061854F82854E83A3E0B40920854F828576
:100F33004E83A3A3E0B40214E550D39404400DAB55
:100F430050AD4DAF4FAE4E1214648036854F82853F
:100F53004E83A3E064097025854F82854E83A3A346
:100F6300E0B40317E550B40412854F82854E83A382
:100F7300A3A3E0FFAD4D126FA580078000AF4D1214
:100F83007A38206803020986C258D26BAF4D125AD1
:100F9300697D607F021277667D327F03127766C2B6
:0F0FA3006BAF4D125A69127091E4786CF6C25E12
:010FB200221C
:083510008F518C528D538B5436
:10351800855382855283A3A3A3E0FF8D828C83E524
:1035280082240412673D8F55E555D3940050030259
:1035380036B1E555942940030236B1E55164067069
:103548004FD26BAF54125A697D527F05127766AF1E
:1035580055124CC4E5532405F582E43552F583E051
:10356800B40112749F2555F582E43406F58374017D
:10357800F07D38800F749F2555F582E43406F58375
:10358800E4F07D367F06127766C26BAF54025A6943
:10359800E5532406F582E43552F583E0640B6003B5
:1035A8000236B1E5532405F582E43552F583E0B4DB
:1035B8000110749F2555F582E43406F5837401F0F3
:1035C800800D749F2555F582E43406F583E4F0E414
:1035D800FFFEE5532407F582E43552F583E5822E94
:1035E800F582E43583F583E0B40B04AF0680040E5E
:1035F800BE08DFEF70030236B1C3940840030236F9
:10360800B175F008E555A424F8F582E5F03400F525
:1036180083EFF07E01EF2401FDE433FCEEC39DEC63
:103628006480F87480985036E5532406F582E435B2
:1036380052F583E5822EF582E43583F583E0FD7546
:10364800F008E555A424F8F582E5F03400F583E5A3
:10365800822EF582E43583F583EDF00E80B7E553CD
:103668002408F582E43552F583E5822FF582E435A6
:1036780083F583E0640B602DEF2408FEC3E5519EBB
:10368800F55175F0041258FAAEF0EE701CE55324AB
:1036980007FDE43552FC7E00ED2FFBEE3CFAAD55FC
:1036A8007F011239EAD26A8002C26AAF54127C0CD6
:0136B80022EF
:10793D008E5CF55DAF5BEF3395E0FEE5592FF5827B
:08794D00E5583EF583A3E0FFBD
:0A795500EFD3940940037F002222C3
:0839EA008F568D578A588B5946
:1039F200755B01E4F55AAF5BEF3395E0FEE5592FB5
:103A0200F582E5583EF583E0FF6409706512795549
:103A1200755C008F5DAE5C7804EF08800633CE33B0
:103A2200CE92E0D8F812793DEF425DAE5CAF5D78A0
:103A320008EF08800633CE33CE92E0D8F88E5CF5DC
:103A42005DAF5BEF3395E0FEE5592FF582E5583E19
:103A5200F583A3A3E0FFE55BFD3395E0FCE5592D7B
:103A6200F582E5583CF583A3A3A3E0FD127A260272
:103A72003B05AF5BEF3395E0FEE5592FF582E55844
:103A82003EF583E0FF127955755C008F5DAE5C7880
:103A920004EF08800633CE33CE92E0D8F812793D97
:103AA200EF425DAE5CAF5D7804EF08800633CE3343
:103AB200CE92E0D8F88E5CF55DAF5BEF3395E0FE19
:103AC200E5592FF582E5583EF583A3A3E0FF12796D
:103AD20055EF425DAE5CAF5D7804EF08800633CEF1
:103AE20033CE92E0D8F88E5CF55DAF5BEF3395E0B4
:103AF200FEE5592FF582E5583EF583A3A3A3E0FF27
:103B0200127955EF425DE556701EAF5AEF3395E0DC
:103B1200FEEF25E0FFEE33FE75F020E557A424D03A
:103B2200F582E5F034068021E556B4012FAF5AEF55
:103B32003395E0FEEF25E0FFEE33FE75F020E5570A
:103B4200A424D0F582E5F03410F583E5822FF582C6
:103B5200E5833EF583E55CF0A3E55DF07404255B47
:103B6200F55B055AC3E55A6480949050030239F814
:013B72002230
:084DC6008F518C528D538B5468
:104DCE00855382855283A3A3A3E0FF8D828C83E556
:104DDE0082240412673D8F55E555D394005003028B
:104DEE004EB3E55594334003024EB3E5516406705D
:104DFE004FD26BAF54125A697D527F05127766AF50
:104E0E0055124CC4E5532405F582E43552F583E082
:104E1E00B40112744F2555F582E43406F5837401FE
:104E2E00F07D38800F744F2555F582E43406F583F6
:104E3E00E4F07D367F06127766C26BAF54025A6974
:104E4E00E5532406F582E43552F583E0640B705584
:104E5E00E5532405F582E43552F583E0B401107470
:104E6E004F2555F582E43406F5837401F0800D74F8
:104E7E004F2555F582E43406F583E4F074F9255197
:104E8E00F55175F0041258FAAFF0EF7014E5532493
:104E9E0006FBE43552FAAD55E4FF1239EAD26A80C8
:104EAE000DC26A8009C26BAF54125A69C26AAF54FE
:034EBE00127C0C57
:014EC10022CE
:023FBA008B5129
:103FBC001267468F54E554D3940050030240FEE53B
:103FCC0054943340030240FED26BAF51125A697DB8
:103FDC00527F05127766AF54124CC4749F2554F56A
:103FEC0082E43406F583E060047D3880027D367F00
:103FFC00061277667F2C7E01127A8D75F008E554D7
:10400C00A424F8F582E5F03400F583E0F55270074E
:10401C007D1B7F061277667D577F02127766E5520D
:10402C0070030240AF755301AF52EF3395E0FEEFD2
:10403C002401FFE43EFEAD53ED3395E0FCC3ED9F50
:10404C00EE6480F8EC6480985059AF53EF3395E0F0
:10405C00FE75F008E554A424F8F582E5F03400F57B
:10406C0083E5822FF582E5833EF583E0FFD3940947
:10407C00400512728F8028AF53EF3395E0FE75F038
:10408C0008E554A424F8F582E5F03400F583E582C4
:10409C002FF582E5833EF583E0FDE4FF127766059C
:1040AC005380857F2C7E01127A8D75F020E554A407
:1040BC0024D0F582E5F03410F583E0FEA3E0FF9008
:1040CC000000EEF0A3EFF04E70077D1B7F06127719
:1040DC00667D0C7F03127766900000E07002A3E00F
:1040EC006009E55414FD7F01122F74C26BAF5102AD
:0940FC005A69C26AAF51127C0C32
:014105002297
:042F74008F558D5692
:102F7800E4F557E555600302301FAF57EF3395E08E
:102F8800FEEF25E0FDEE33FCAF56EF3395E0FEEFA4
:102F98007805C333CE33CED8F924F0F58274063ED3
:102FA800F583E5822DF582E5833CF583E0FAA3E01D
:102FB800FB780CFFAE02088006A2E0CE13CE13D831
:102FC800F8540FF5587808AF03AE02EF088006A250
:102FD800E0CE13CE13D8F8540FF559AF56EF33950A
:102FE800E0FEEF7805C333CE33CED8F924F0F5826E
:102FF80074063EF583E5822DF582E5833CF583E092
:10300800FCA3E0FD7804FFAE04088006A2E0CE131E
:10301800CE13D8F80230C2E555640160030230CB04
:10302800AF57EF3395E0FEEF25E0FDEE33FCAF56EA
:10303800EF3395E0FEEF7805C333CE33CED8F924CD
:10304800F0F58274103EF583E5822DF582E5833C28
:10305800F583E0FAA3E0FB780CFFAE02088006A235
:10306800E0CE13CE13D8F8540FF5587808AF03AE56
:1030780002EF088006A2E0CE13CE13D8F8540FF55D
:1030880059AF56EF3395E0FEEF7805C333CE33CE14
:10309800D8F924F0F58274103EF583E5822DF58287
:1030A800E5833CF583E0FCA3E0FD7804FFAE04086B
:1030B8008006A2E0CE13CE13D8F8540FF55AED547B
:1030C8000FF55BE558700FE559700BE55A7007E589
:1030D8005B700302315DAD58E4FF127766AD59E4C9
:1030E800FF127766E55864097048855A5CAF5CFE44
:1030F8007804EF08800633CE33CE92E0D8F8F55C3A
:10310800E55B425CE55CB4990B7D09E4FF127766E8
:103118007D098027E55C75F00A84F55DFDE4FF1202
:103128007766E55D75F00AA4FFC3E55C9FF55DFD74
:103138008009AD5AE4FF127766AD5BE4FF1277664B
:103148007FF47E01127A8D0557C3E557648094A0F9
:053158005003022F7B73
:01315D00224F
:025C78008B514E
:105C7A001267468F52E552D394005003025D14E531
:105C8A005294334003025D14D26BAF51125A697DAC
:105C9A00527F05127766AF52124CC4744F2552F5E3
:105CAA0082E43406F583E060047D3880027D367F25
:105CBA00061277667F2C7E01127A8D7F2C7E011266
:105CCA007A8D75F020E552A424D0F582E5F03406E9
:105CDA00F583E0FEA3E0FF900000EEF0A3EFF04EA4
:105CEA0070077D1B7F061277667D0C7F031277662D
:105CFA00900000E07002A3E06009E55214FDE4FFA1
:105D0A00122F74C26BAF51025A69C26AAF51127C28
:015D1A000C7C
:015D1B002265
:026589008B5134
:10658B00126746AD07EDD39400406BED9433506624
:10659B00E4FCECFF3395E0FEEF25E0FFEE33FE75F8
:1065AB00F020EDA424D0F582E5F03410F583E582DC
:1065BB002FF582E5833EF583E4F0A3F00CBC10D2FB
:1065CB00749F2DF582E43406F583E4F0FCECFF3385
:1065DB0095E0FE75F008EDA424F8F582E5F03400A3
:1065EB00F583E5822FF582E5833EF583E4F00CBC61
:0D65FB0008DBD26A8002C26AAF51127C0C2C
:01660800226F
:026B57008B5160
:106B5900126746AD07EDD394004045ED943350409C
:106B6900E4FCECFF3395E0FEEF25E0FFEE33FE7524
:106B7900F020EDA424D0F582E5F03406F583E58212
:106B89002FF582E5833EF583E4F0A3F00CBC10D227
:106B9900744F2DF582E43406F583E4F0D26A80025D
:076BA900C26AAF51127C0C1F
:016BB00022C2
:1075C3002430F58274003EF583EDF0AF55EF33952B
:1075D300E0FEE5522FF582E5513EF583A3A3E0FFDC
:1075E300D3EF648094814008EF6480948A50012231
:0375F3007F0022F4
:107BB500D3EF648094804008EF648094A150012243
:037BC5007F00221C
:081464008E518F528D538B5401
:10146C008F828E83A3A3A3E014F55674FC2554F548
:10147C00546403600FE55464076009E554640B6021
:10148C0003021807C3E556648094805003021807C2
:10149C00E556648094884003021807E4F555AF566E
:1014AC00EF3395E0FEEF7803C333CE33CED8F92477
:1014BC0030F58274003EF583AF55EF3395E0FEE5D1
:1014CC00822FF582E5833EF583E4F00555E555B4AE
:1014DC0008CC755504E5546403705FAF55EF339534
:1014EC00E0FEE5522FF582E5513EF583E0FFE55530
:1014FC00FD3395E0FCE5522DF582E5513CF583A3D7
:10150C00E0FD126746127BB5AD07AF56EF3395E0A1
:10151C00FEEF7803C333CE33CED8F91275C3AD07C3
:10152C00AF56EF3395E0FEEF7803C333CE33CED80E
:10153C00F92431F58274000217FEE5546407600348
:10154C00021639AF55EF3395E0FEE5522FF582E5E3
:10155C00513EF583E0FFE555FD3395E0FCE5522D5A
:10156C00F582E5513CF583A3E0FD126746127BB58D
:10157C00AD07AF56EF3395E0FEEF7803C333CE33B0
:10158C00CED8F91275C3AD07AF56EF3395E0FEEF29
:10159C007803C333CE33CED8F92431F58274003EB0
:1015AC00F583EDF0AF55EF3395E0FEE5522FF58264
:1015BC00E5513EF583A31275DFAD07AF56EF3395BA
:1015CC00E0FEEF7803C333CE33CED8F91266FF12A8
:1015DC007BB5AD07AF56EF3395E0FEEF7803C33321
:1015EC00CE33CED8F92433F58274003EF583EDF07A
:1015FC00AF55EF3395E0FEE5522FF582E5513EF500
:10160C0083E5822406F582E43583F583E0FF1275C9
:10161C00E3AD07AF56EF3395E0FEEF7803C333CE5F
:10162C0033CED8F92434F58274000217FEE55464E5
:10163C000B6003021807AF55EF3395E0FEE5522F10
:10164C00F582E5513EF583E0FFE555FD3395E0FC71
:10165C00E5522DF582E5513CF583A3E0FD1267467A
:10166C00127BB5AD07AF56EF3395E0FEEF7803C3B1
:10167C0033CE33CED8F91275C3AD07AF56EF3395D1
:10168C00E0FEEF7803C333CE33CED8F92431F582A4
:10169C0074003EF583EDF0AF55EF3395E0FEE55267
:1016AC002FF582E5513EF583A31275DFAD07AF56DA
:1016BC00EF3395E0FEEF7803C333CE33CED8F91277
:1016CC0066FF127BB5AD07AF56EF3395E0FEEF78B2
:1016DC0003C333CE33CED8F92433F58274003EF5F0
:1016EC0083EDF0AF55EF3395E0FEE5522FF582E533
:1016FC00513EF583E5822406F582E43583F583E0DB
:10170C00FF1275E3AD07AF56EF3395E0FEEF7803AC
:10171C00C333CE33CED8F92434F58274003EF5832E
:10172C00EDF0AF55EF3395E0FEE5522FF582E55124
:10173C003EF583E5822407F582E43583F583E0FFEB
:10174C001275E3AD07AF56EF3395E0FEEF7803C3A8
:10175C0033CE33CED8F92435F58274003EF583EDC3
:10176C00F0AF55EF3395E0FEE5522FF582E5513E93
:10177C00F583E5822408F582E43583F583E0FFE503
:10178C0055FD3395E0FCE5522DF582E5513CF58392
:10179C00E582240912673D127BB5AD07AF56EF33D6
:1017AC0095E0FEEF7803C333CE33CED8F92436F56B
:1017BC008274003EF583EDF0AF55EF3395E0FEE516
:1017CC00522FF582E5513EF583E582240AF582E439
:1017DC003583F583E0FF1275E3AD07AF56EF339514
:1017EC00E0FEEF7803C333CE33CED8F92437F5823D
:1017FC0074003EF583EDF0D26A8002C26AAF5312D8
:02180C007C0C52
:01180E0022B7
:1070DC00EF24FE601014601314601624037016D293
:1070EC0008D2248010D209D225800AD20ED2268052
:1070FC0004D20CD2277FF47E01127A8D753D04E503
:10710C003D70FC7F647E00127A8DC224C225C2269B
:0B711C00C227C208C209C20EC20C222A
:0456BB008D51AC075A
:1056BF00C3EC64809481500302577EEC648094891C
:1056CF00400302577EE4F552AF51EF3395E0FEEF02
:1056DF007803C333CE33CED8F924E8F582741A3E5B
:1056EF00F583AF52EF3395E0FEE5822FF582E58328
:1056FF003EF583E0FD74182FF582741D3EF583EDA2
:10570F00F00552E552B408C0EC14FFAD51127249C6
:10571F00D269AF51125B1D753D017F327E00127A47
:10572F008DE53D70FCC269AF51125B1DE4F552E58A
:10573F0052FD3395E0FC74182DF582741D3CF583F2
:10574F00E0FBAF51EF3395E0FEEF7803C333CE3379
:10575F00CED8F924E8F582741A3EF583E5822DF54B
:0F576F0082E5833CF583EBF00552E552B408C0A8
:01577E002208
:046FA5008D51AC0757
:106FA900D3EC64809480403CEC648094895035E44F
:106FB900FDECFF3395E0FEEF7803C333CE33CED833
:106FC900F92428F58274003EF583EDFF3395E0FE40
:106FD900E5822FF582E5833EF583E4F00DBD08D106
:0B6FE900D26A8002C26AAF51127C0C19
:016FF400227A
:044789008C528D536E
:10478D00D3EF648094805003024891EF6480949538
:10479D004003024891EB648094875003024891EBEB
:1047AD00648094E44003024891EF3395E0FEEF7886
:1047BD0005C333CE33CED8F92460F58274033EAFF2
:1047CD0082F5568F57EB24FBF558D3940250030214
:1047DD004891E55875F00384E5F06003024891E5D2
:1047ED005875F00384F55AC394104003024891059F
:1047FD0057E557AE567002055614F5828E83E55A6D
:10480D00F074052553F553E43552F552E4F558E5AA
:10481D0058C3955A506A855382855283E0F559B431
:10482D000A130557E557AE567002055614F5828EDC
:10483D0083E4F080120557E557AE56700205561405
:10484D00F5828E83E559F0855382855283A3E0FF6F
:10485D00855382855283A3A3E0FD127A268F5905D5
:10486D0057E557AE567002055614F5828E83E559FD
:10487D00F074032553F553E43552F5520558808FE6
:0B488D00D26A8002C26AAF55127C0C98
:0148980022FD
:04577F008F518D5267
:10578300E551D394005003025836E5519415400374
:10579300025836D26BAF52125A697D5F7F0512777A
:1057A30066AD51E4FF1277667D527F041277667F00
:1057B300F47E01127A8D75F020E551A42460F58200
:1057C300E5F03403AF82F5558F56F583E0F553606A
:1057D3004DD394004056E55394105050E55325E0C3
:1057E300F553755401E5532401FFE433FEC3E55437
:1057F3009FEE6480F87480985032E5562554F58204
:10580300E43555F583E0FFE5562554F582E4355537
:10581300F583A3E0FD1277660554055480C77D1B0D
:105823007F061277667D5F7F05127766C26BAF5284
:0A583300025A69C26AAF52127C0CDF
:01583D002248
:10780B008D51EFD3940A4006EFD3940F4003EF70E2
:10781B000E90063FEFF0D26AAF51127C0CD322C20E
:08782B006AAF51127C0CC3226C
:107833008D51EFD3940A4006EFD3940F4003EF70BA
:107843000E90063BEFF0D26AAF51127C0CD322C2EA
:087853006AAF51127C0CC32244
:10728F008F55E555B40B067D5F7F078034E555B408
:10729F000C067D5E7F068029E555B40D067D0A7FBD
:1072AF0002801EE555B40E067D327F028013E55530
:1072BF00B40F067D467F028008E55570077D0A7F73
:0572CF000312776622A6
:10770E008F51D26B125A697D207F051277667D2EBE
:10771E007F031277667D527F0412776690063FE0F4
:0C772E00FF12728FC26BAF51125A692219
:10773A008F51D26B125A697D207F051277667D219F
:10774A007F061277667D527F0412776690063BE0C9
:0C775A00FF12728FC26BAF51125A6922ED
:1079A0008D51D3EF64809480400EEF6480948650B4
:1079B00007127527D26A8002C26AAF51127C0C226C
:06744E008D51AB07AA06F8
:107454008B828A83A3A3A3E0FFEB2404F582E43A9E
:10746400126742D3EF648094804010EF648094A14B
:10747400500990063DEFF0D26A8002C26AAF511201
:027484007C0C7E
:0174860022E3
:067628008D51AB07AA061C
:10762E008B828A83A3A3A3E0FFEB2404F582E43AC2
:10763E00126742EFC39421500990063CEFF0D26AD4
:09764E008002C26AAF51127C0CEB
:017657002210
:065F00008E518F528B53FD
:105F0600755406755540D3ED64809484407CED64E9
:105F16008094A55075ED24FDF556D39404406BE5A9
:105F26005620E06613F5570555E555AE5470020543
:105F36005414F5828E83E557F074032552F552E426
:105F46003551F551E4F556E556C39557503385520C
:105F560082855183E0FFA3E0FD127A260555E555BB
:105F6600AC547002055414F5828C83EFF00552E5AB
:105F760052700205510552E55270020551055680D0
:105F8600C6D26AAF53127C0CD322C26AAF53127CBC
:025F96000CC33A
:015F980022E6
:084899008E518F528D538B5498
:1048A100C269D3E55364809484500302494EE553B1
:1048B1006480948D400302494E8F828E83A3A3E0CE
:1048C100640A600302494E8F828E83A3A3A3E0147E
:1048D100B4080050769048E475F003A4C58325F030
:1048E100C583730248FC02490602491002491A02B3
:1048F100492402492E02493802494275550075562C
:1049010080D2698048755500755688D269803E7598
:104911005500755690D2698034755500755698D2F8
:1049210069802A7555007556A0D269802075550099
:104931007556A8D26980167555007556B0D2698032
:104941000C755500755678D2698002C2693069507C
:10495100E4FFEF7C002556FDEC35558D82F583E4AF
:10496100F00FBF08EDE55324FB855682855583F092
:104971007F01E5522404F582E43551F583E5822F68
:10498100F582E43583F583E0FEEF7C002556FDECEE
:1049910035558D82F583EEF00FBF08D6D26A8002BD
:0749A100C26AAF54127C0C46
:0149A80022EC
:0461E8008E548F55ED
:1061EC000555E5557002055414F5828E83E0F5577C
:1061FC006074C39408506F7F2C7E01127A8DE4F585
:10620C0056E556C39557505E855582855483E0609C
:10621C003624F5601414601714601A14601D146091
:10622C002024057028E4FD802D7D5F7F0780287D6C
:10623C005E7F0680227D0A7F02801C7D327F028079
:10624C00167D467F0280107D0A7F03800A85558269
:10625C00855483E0FDE4FF1277660555E555700221
:06626C0005540556809B5D
:016272002209
:022D80008B5175
:102D8200C269EF640A6003022F5BED14B4080040CD
:102D920003022F59902DA475F003A4C58325F0C515
:102DA2008373022DBC022DF0022E24022E58022E15
:102DB2008C022EC0022EF3022F26D26BAF51125A72
:102DC200697D577F021277667D05E4FF127766E41C
:102DD200FDFF1277667D01E4FF1277667D527F0464
:102DE200127766755200755380D269022F5BD26BDF
:102DF200AF51125A697D577F021277667D05E4FF53
:102E0200127766E4FDFF1277667D02E4FF127766B1
:102E12007D527F04127766755200755388D269021B
:102E22002F5BD26BAF51125A697D577F02127766C0
:102E32007D05E4FF127766E4FDFF1277667D03E409
:102E4200FF1277667D527F041277667552007553C2
:102E520090D269022F5BD26BAF51125A697D577FB4
:102E6200021277667D05E4FF127766E4FDFF1277B2
:102E7200667D04E4FF1277667D527F0412776675E1
:102E82005200755398D269022F5BD26BAF51125A1E
:102E9200697D577F021277667D05E4FF127766E44B
:102EA200FDFF1277667D05E4FF1277667D527F048F
:102EB2001277667552007553A0D269022F5BD26BEE
:102EC200AF51125A697D577F021277667D05E4FF82
:102ED200127766E4FDFF1277667D06E4FF127766DD
:102EE2007D527F041277667552007553A8D26980AD
:102EF20068D26BAF51125A697D577F021277667D95
:102F020005E4FF127766E4FDFF1277667D07E4FFB2
:102F12001277667D527F041277667552007553B040
:102F2200D2698035D26BAF51125A697D577F021236
:102F320077667D05E4FF127766E4FDFF1277667D12
:102F420008E4FF1277667D527F041277667552009D
:102F5200755378D2698002C269306909AF53AE52A3
:102F62001261E88005AF51127A38C26BAF51125A22
:012F720069F5
:012F7300223B
:08315E008E518F528D538B54EA
:10316600C2698F828E83A3A3E0640A6003023215CC
:10317600124BBD8E568F57D3E557943BE5569400B8
:103186005003023210E5579408E5569407507BC366
:10319600E5536480948A5072855282855183A3A335
:1031A600A3E0F555B401069006000232BBE555B41E
:1031B60002069006020232BBE555B40306900604E9
:1031C6000232BBE555B404069006060232BBE5554D
:1031D600B405069006080232BBE555B4060690060D
:1031E6000A0232BBE555B4070690060C0232BBE56F
:1031F60055B4080690060E0232BBE555B409069092
:1032060006100232BBD269023337D26902333785E0
:103216005282855183A3A3E0640160030232C5ADE7
:1032260053AF52AE51124BBD8E568F57D3E55794BE
:103236003BE55694005003023337E5579408E556AC
:1032460094074003023337C3E5536480948A4003EE
:10325600023337855282855183A3A3A3E0F555B483
:103266000A05900612804EE555B4010590061480B5
:1032760044E555B40205900616803AE555B40305B3
:103286009006188030E555B4040590061A8026E5A8
:1032960055B4050590061C801CE555B40605900638
:1032A6001E8012E555B407059006208008E555B442
:1032B6000809900622E556F0A3806FD269807285D0
:1032C6005282855183A3A3E064027065AD53AF5269
:1032D600AE51126BB17556008F57C3E5579463E52F
:1032E600569400504CC3E5536480948850438552ED
:1032F60082855183A3A3A3E0F555B4010790063058
:10330600EFF0802DE555B40205900631801CE55599
:10331600B403059006328012E555B40405900633D1
:103326008008E555B40508900634E557F08002D2CA
:0F33360069306904C26A8002D26AAF54127C0CFB
:013345002265
:10267D008F518D528B53E551640A6003022729E572
:10268D0052C3940A40030228FFD26BAF53125A690A
:10269D007D277F081277667D06E4FF127766E4FDDD
:1026AD00FF127766AD52E4FF1277667D527F0412FA
:1026BD007766E55214B4090040030228F89026D835
:1026CD0075F003A4C58325F0C583730226F3022696
:1026DD00F90226FF02270502270B022711022717F1
:1026ED0002271D02272390060002283990060202B8
:1026FD0028399006040228399006060228399006DA
:10270D000802283990060A02283990060C02283949
:10271D0090060E022839900610022839E551640101
:10272D006003022847E552D394004006E552940910
:10273D004009E552640A6003022844D26BAF53127C
:10274D005A697D277F081277667D06E4FF1277664A
:10275D00E552B40A147D0AE4FF1277667D527F04B8
:10276D00127766900612022839E552B401147D0BDA
:10277D00E4FF1277667D527F04127766900614028D
:10278D002839E552B402147D0CE4FF1277667D52B0
:10279D007F04127766900616022839E552B40313AA
:1027AD007D0DE4FF1277667D527F041277669006E9
:1027BD00188079E552B404137D0EE4FF1277667D1F
:1027CD00527F0412776690061A8061E552B40513A4
:1027DD007D0FE4FF1277667D527F041277669006B7
:1027ED001C8049E552B406137D10E4FF1277667D17
:1027FD00527F0412776690061E8031E552B407139E
:10280D007D11E4FF1277667D527F04127766900684
:10281D00208019E552640860030229067D12FF121B
:10282D0077667D527F04127766900622E0FEA3E064
:10283D00FF1274F20229060228FFE55164026003BB
:10284D00022906E552D3940050030228FFE5529465
:10285D000740030228FFD26BAF53125A697D277FC1
:10286D00081277667D06E4FF1277667D14E4FF1289
:10287D007766E55224FE60201460301460401460C9
:10288D0050240470667D01E4FF1277667D527F044B
:10289D00127766900630804A7D02E4FF1277667DDE
:1028AD00527F0412776690063180377D03E4FF1264
:1028BD0077667D527F0412776690063280247D0400
:1028CD00E4FF1277667D527F04127766900633809F
:1028DD00117D05E4FF1277667D527F0412776690B5
:1028ED000634E0FF7E00127658800EAF53127A3810
:1028FD008007C26AAF53127C0CC26BAF53125A6978
:01290D0022A7
:064BBD008E588F59A90576
:104BC3007D057C00E5592DF582E5583CF583E0C36E
:104BD300940A400CE5592DF582E5583CF583E4F041
:104BE3000DBD00010CED640A4C70D9B90610E559EE
:104BF3002405F582E43558F583E0FF7E0022E9645D
:104C0300077019E5592405F582E43558F583E075F5
:104C1300F00AA4ACF0FDE55924068032E96408707B
:104C23003DE5592405F582E43558F583E075F064D4
:104C3300A4ACF0FDE5592406F582E43558F583E08C
:104C430075F00AA42DFDE5F03CFCE5592407F58237
:104C5300E43558F583E02DFDE43CAF05FE22E9641D
:104C630009705AE5592405F582E43558F583E0FFC8
:104C73007E007C037DE812591CAC06AD07E5592480
:104C830006F582E43558F583E075F064A42DFDE55F
:104C9300F03CFCE5592407F582E43558F583E075CB
:104CA300F00AA42DFDE5F03CFCE5592408F582E467
:104CB3003558F583E02DFDE43CFEAF0522E4FEFF0D
:014CC30022CE
:066BB1008E588F59A90562
:106BB7007F057E00E5592FF582E5583EF583E0C352
:106BC700940A400CE5592FF582E5583EF583E4F029
:106BD7000FBF00010EEF64084E70D9E964077020FB
:106BE700E5592405F582E43558F583E075F00AA4E4
:106BF700FFE5592406F582E43558F583E02FFF2297
:026C07007F000C
:016C09002268
:104CC4008F56E556D3945940147D5AE4FF12776603
:104CD400E55624A6FD7003024DC5024DC0E556D32A
:104CE400944F401AE556945A50147D50E4FF1277BD
:104CF40066E55624B0FD7003024DC5024DC0E5566D
:104D0400D39445401AE556945050147D46E4FF125E
:104D14007766E55624BAFD7003024DC5024DC0E521
:104D240056D3943B4019E556944650137D3CE4FF1A
:104D3400127766E55624C4FD7003024DC5807DE5F7
:104D440056D394314016E556943C50107D32E4FF1E
:104D5400127766E55624CEFD60678060E556D394ED
:104D6400274016E556943250107D28E4FF127766EA
:104D7400E55624D8FD604A8043E556D3941D401679
:104D8400E556942850107D1EE4FF127766E55624FC
:104D9400E2FD602D8026E556D394134016E5569423
:104DA4001E50107D14E4FF127766E55624ECFD6076
:104DB400108009E556C394145007AD56E4FF1277EA
:024DC400662265
:107658008E548F557C007D0A12592EAD07E4FF1217
:1076680077667D5B7F06127766AE54AF557C007DEA
:107678000A12592EE4FF1277667D4A7F0702776661
:0474F2008E548F55D0
:1074F6007C007D3C12592EAA06AB07124CC47D05B2
:107506007F06127766AE54AF557C007D3C12592E2D
:10751600ED4C600CAF05124CC47D4A7F07127766AE
:017526002242
:027127008D5188
:10712900D3EF648094804038EF648094955031EFB8
:107139003395E0FEEF7805C333CE33CED8F924601A
:10714900F58274033EAF82FEE4FD0FEFAA067001DB
:107159000E14F5828A83E4F00DBD20EED26A800216
:07716900C26AAF51127C0C59
:0171700022FC
:1073D5008F51900640E0D394024015D269125B1D8F
:1073E500753D037F327E00127A8DE53D70FC801578
:1073F500D269AF51125B1D7D1B7F061277667D0C2E
:0D7405007F03127766C269AF51125B1D2232
:107BDA007E10900640E4F0A3DEFC7E10D26A127C8E
:017BEA000C8E
:017BEB002277
:107919008F5CD26B125A697D607F021277667D3265
:107929007F061277667D1E7F05127766C26BAF5C94
:04793900125A692253
:107A38008F5CD26B125A697D607F021277667D3047
:0D7A48007F03127766C26BAF5C125A692291
:0E7C0C008F5B306A03027919AF5B127A38225F
:1066FF002432F58274003EF583EDF0AF55EF3395FC
:10670F00E0FEE5522FF582E5513EF583E582240444
:10671F00F582E43583F583E0FFE555FD3395E0FC25
:10672F00E5522DF582E5513CF583E5822405F5828E
:07673F00E43583F583E0FD62
:10674600EFD394004015EF940B5010EFC3940A500A
:1067560008EF75F00AA4FE8002E4FEEDD394004033
:106766000EED940B5009EDC3940A5003ED2EFEAFC7
:01677600061C
:0167770022FF
:03000000027BFD83
:0F7BFD00758E0078FEE4F6D8FD75816C0255EFA9
:107B2400D292C0F075F008C29100A29233D291D5DE
:067B3400F0F5D0F0FF2285
:107B3A00EFC0F075F00833C291929333D291D5F029
:067B4A00F6D0F0C291220A
:10776600EFFEEDFF1280008E2F8F30125D1C755FCD
:1077760064AF5F155FEFD39400400EE4F55EE55EFF
:09778600C3943A50EC055E80F555
:01778F0022D7
:105D1C00D2A885A86175A881C244853082852F835D
:105D2C00E493F560C4540FF5604360F0856080C265
:105D3C0084D28500C2870000D287007580FF7580F1
:105D4C00FEC284C28500C28700000000D2870075A5
:105D5C0080FFD24475623E756380E4F56030941D1B
:105D6C000560E560B464F6123346E56315637002B2
:105D7C001562D3E5639400E562940050DD75623ED4
:105D8C00756380E4F56020941D0560E560B464F6ED
:105D9C00123346E563156370021562D3E563940014
:105DAC00E562940050DD8561A8C2A87F147E0012C4
:025DBC007A8DDE
:015DBE0022C2
:107790007580FDC284C28500C28700000000D287C8
:1077A000007580FF7F147E00127A8D7F997E09120A
:0A77B00080008E2F8F30125D1C2226
:1058FA00C2D530F707B2D563F0FF05F030E70CB236
:10590A00D5F4048463F0FF05F080018430D502F4F5
:02591A00042265
:10591C00EF8DF0A4A8F0CF8CF0A428CE8DF0A42E9F
:02592C00FE2259
:10592E00BC000BBE0029EF8DF084FFADF022E4CC5D
:10593E00F875F008EF2FFFEE33FEEC33FCEE9DEC26
:10594E00984005FCEE9DFE0FD5F0E9E4CEFD22ED6C
:10595E00F8F5F0EE8420D21CFEADF075F008EF2FB6
:10596E00FFED33FD4007985006D5F0F222C398FDA7
:05597E000FD5F0EA2244
:10598300EB9FF5F0EA9E42F0E99D42F0E89C45F07A
:0159930022F1
:105994007401FF3395E0FEFDFC080808E6CF2FF6FE
:1059A40018E6CE3EF618E6CD3DF618E6CC3CF622D7
:107BEC00EFC39461400AEF947B5005EF24E0FF2231
:017BFC002266
:00000001FF
